S02000006F70656E626C745F6F6C696D65785F73746D3332703430352E7372656302
S31508000000E0080020297B0008857B0008897B00081A
S315080000108D7B0008917B0008957B00080000000096
S31508000020000000000000000000000000997B0008A6
S315080000309D7B000800000000A17B0008A57B000846
S31508000040A97B0008AD7B0008B17B0008B57B0008DA
S31508000050B97B0008BD7B0008C17B0008C57B00088A
S31508000060C97B0008CD7B0008D17B0008D57B00083A
S31508000070D97B0008DD7B0008E17B0008E57B0008EA
S31508000080E97B0008ED7B0008F17B0008F57B00089A
S31508000090F97B0008FD7B0008017C0008057C000848
S315080000A0097C00080D7C0008117C0008157C0008F6
S315080000B0197C00081D7C0008217C0008257C0008A6
S315080000C0297C00082D7C0008317C0008357C000856
S315080000D0397C00083D7C0008417C0008457C000806
S315080000E0497C00084D7C0008517C0008557C0008B6
S315080000F0597C00085D7C0008617C0008657C000866
S31508000100697C00086D7C0008717C0008757C000815
S31508000110797C00087D7C0008817C0008857C0008C5
S31508000120897C00088D7C0008917C0008957C000875
S31508000130997C00089D7C0008A17C0008A57C000825
S31508000140A97C0008AD7C0008B17C0008B57C0008D5
S31508000150B97C0008BD7C0008C17C0008C57C000885
S31508000160C97C0008CD7C0008D17C0008D57C000835
S31508000170D97C0008DD7C0008E17C0008E57C0008E5
S31508000180E97C0008ED7C00084178007850EA0121F6
S31508000190080080B27047C178827852EA0121427815
S315080001A052EA0121007850EA0121080070470170DF
S315080001B0401C89B2090A0170401C70470170401C36
S315080001C0090A0170401C090A0170401C090A0170DD
S315080001D0401C7047002A06D00B780370491C401C47
S315080001E0521E002AF8D170470170401C521E002A80
S315080001F0FAD1704710B4002303780C781B1B491CEE
S31508000200401C521E002A01D0002BF5D0180010BC45
S31508000210704700E0401C0278002A02D002788A4221
S31508000220F8D100787047F8B505000024E87800286A
S3150800023020D0EE6A0123320015F13001687802F009
S315080002402AFA002801D0012414E00020E870286A60
S31508000250301AA96988420DD2AF7809E0A8698619CB
S315080002600123320015F13001687802F014FA7F1E76
S31508000270022FF3D22000C0B2F2BD70B504000D0003
S315080002800026E06A854213D02000FFF7CCFF06005F
S31508000290F6B2002E0CD101232A0014F13001607841
S315080002A002F0B0F9002802D05FF0FF350126E562BA
S315080002B03000C0B270BD38B504002000FFF7B3FFA8
S315080002C00500EDB2002D3FD12078032834D12079DE
S315080002D0012831D14FF40072002114F13000FFF7E4
S315080002E083FF4AF6552104F22E20FFF760FFDFF858
S315080002F0B41714F13000FFF761FFDFF8AC174FF4BD
S3150800030005702044FFF75AFF21694FF40670204410
S31508000310FFF754FFE1684FF407702044FFF74EFFDC
S31508000320E069401CE0620123E26A14F1300160785A
S3150800033002F0B1F90020207100220021607802F055
S3150800034003FA002800D001252800C0B232BD891E54
S315080003504269921E914201D3002003E04289806AD5
S3150800036002FB010070472DE9F0410C000568022CDC
S3150800037002D36869844201D3012656E05FF0FF364E
S315080003802878012804D04FD303283BD029D34BE043
S31508000390270017EB5707286A10EB57212800FFF7A5
S315080003A06CFF002841D1F805C00D284490F830802C
S315080003B07F1C286A10EB57212800FFF75EFF0028EC
S315080003C033D1F805C00D284490F8300058EA0028C3
S315080003D0E00702D55FEA181602E05FEA0856360D0E
S315080003E023E0286A10EB14212800FFF746FF0028AF
S315080003F01BD16000C005C00D28443030FFF7C4FE8D
S31508000400060012E0286A10EBD4112800FFF735FF22
S3150800041000280AD1A000C005C00D28443030FFF7D7
S31508000420BAFE20F0704600E001263000BDE8F081F3
S315080004302DE9F04104000D0016000227022D7CD399
S315080004406069854279D22078012804D075D30328BB
S3150800045055D03ED371E0A84618EB5808206A10EB31
S3150800046058212000FFF709FF0700FFB2002F64D1CB
S315080004705FEAC850C00D2044303018F10108E9077A
S3150800048005D5017811F00F0151EA061100E0310097
S3150800049001700120E070206A10EB58212000FFF758
S315080004A0ECFE0700FFB2002F47D15FEAC850C00D27
S315080004B020443030E90701D5310906E0017811F00A
S315080004C0F001320A12F00F02114301700120E070A8
S315080004D033E0206A10EB15212000FFF7CEFE070057
S315080004E0FFB2002F29D1310089B26800C005C00DBE
S315080004F020443030FFF75BFE0120E0701DE0206AE3
S3150800050010EBD5112000FFF7B8FE0700FFB2002F49
S3150800051013D1A800C005C00D20443030FFF73BFEBC
S31508000520000F60F31F763100A800C005C00D2044F7
S315080005303030FFF743FE0120E0703800C0B2BDE856
S31508000540F081F8B504000F00110000202568022F7D
S3150800055002D36869874201D3022035E0002909D011
S315080005605FF0FF322800FFF763FFC0B2002801D012
S31508000570C0B229E039002000FFF7F5FE0600002E7C
S3150800058021D0012E01D102201EE016F1010F01D162
S31508000590012019E0002239002800FFF749FFC0B200
S315080005A0002801D0C0B20FE0286910F1010F06D06B
S315080005B02869401C2861287950F001002871370005
S315080005C068698742D6D30020F2BD2DE9F0410700BD
S315080005D00C003D68002C0AD1D5F80C80B8F1000F44
S315080005E002D06869804511D35FF001080EE021004A
S315080005F03800FFF7B8FE022801D2012049E010F1C1
S31508000600010F46D06969884243D3A0464646761C00
S315080006106869864204D30226B04501D2002038E034
S3150800062031003800FFF79FFE002820D15FF0FF3227
S3150800063031002800FFF7FCFEC0B2002806D1002CC6
S3150800064004D0320021002800FFF7F2FEC0B20028CD
S3150800065017D1EE6028696969891E884202D228691D
S31508000660401E2861287950F00100287110E0012801
S3150800067002D010F1010F00D10BE04645C7D100208A
S3150800068007E0C0B2012802D15FF0FF3600E001267C
S315080006903000BDE8F0812DE9F04104000D0027681F
S315080006A0B5F5001F02D215F01F0F01D0022042E057
S315080006B02561A668002E03D13878032800DB7E6AF8
S315080006C0002E08D168093989884201D3022032E010
S315080006D0786AA0611FE078894FF4007101FB00F881
S315080006E001E0B5EB0805454510D331002000FFF7BA
S315080006F03AFE060016F1010F01D101201BE0022E79
S3150800070002D378698642ECD3022014E0310038001F
S31508000710FFF71DFEA0616661A069002801D10220CD
S3150800072009E0A06910EB5520A061E805C00D384422
S315080007303030E0610020BDE8F0812DE9F041040089
S315080007400E002568206910F12007A069002802D04C
S31508000750B7F5001F01D3042076E0F8056DD1A0692E
S31508000760401CA0616069002807D178092989884258
S3150800077063D30020A061042066E06889401E10EA61
S31508000780572F5AD161692000FFF7EDFD8046B8F171
S31508000790020F01D2022057E018F1010F01D1012002
S315080007A052E06869804541D3002E03D10020A0613C
S315080007B0042049E061692000FFF707FF8046B8F189
S315080007C0000F01D107203FE0B8F1010F01D1022047
S315080007D03AE018F1010F01D1012035E02800FFF7B2
S315080007E022FD002801D001202EE04FF400720021DE
S315080007F015F13000FFF7F8FC002641462800FFF700
S31508000800A6FDE86203E0761CE86A401CE86268898F
S31508000810864208D20120E8702800FFF704FD002868
S31508000820F1D0012010E0E86A801BE862C4F8148061
S3150800083041462800FFF78BFDA0612761F805C00D2A
S3150800084028443030E0610020BDE8F081F8B50400A6
S315080008500D00276800212000FFF71DFFC0B2002801
S315080008601BD10026A1693800FFF707FDC0B2002892
S3150800087013D1E1690978E52903D0E16909780029E6
S3150800088003D1761CAE4201D107E0002601212000E3
S31508000890FFF753FFC0B20028E4D0C0B2042800D145
S315080008A00720C0B2F2BD70B504000D0015F11A009C
S315080008B0FFF76AFC06002078032805D115F1140015
S315080008C0FFF762FC56EA0046300070BD70B50400BA
S315080008D00D001600310089B215F11A00FFF767FC02
S315080008E02078032805D1310C89B215F11400FFF7D9
S315080008F05EFC70BD2DE9F84304000D0015F11A00E1
S31508000900FFF742FC002801D0002044E0287810F0C8
S315080009103F00401E0D2101FB00F65FF0010800278D
S3150800092014E0FF2E0ED2484680B202F064F88046E4
S3150800093034F8160002F05FF8761C1FFA88F880B2C1
S31508000940804501D0002026E0C8467F1C0D2F13D213
S31508000950DFF81C0DC05D2844FFF716FC81461FFA18
S3150800096088F8B8F1000FDCD11FFA89F94FF6FF7045
S315080009708145EAD000200EE0287840060AD51FFAFD
S3150800098088F8B8F1000F05D034F81600002801D011
S31508000990002000E00120BDE8F2832DE9F0410400C3
S315080009A00D0015F11A00FFF7EFFB002801D0002013
S315080009B032E0287810F03F00401E0D2101FB00F6BA
S315080009C05FF00108002708E0FF2E01D3002023E08E
S315080009D0804624F81680761C7F1C0D2F11D2DFF86E
S315080009E0900CC05D2844FFF7CFFB1FFA88F8B8F1D2
S315080009F0000FE9D180B24FF6FF718842ECD0002093
S31508000A000AE02878400606D5FF2E01D3002003E029
S31508000A10002024F816000120BDE8F0812DE9F843EE
S31508000A2004000D0016006B730F20E872002028736F
S31508000A30002115F11A00FFF7BAFBF6B2701E0D2158
S31508000A4001FB00F95FF000081FFA88F847461FFA0D
S31508000A5088F84FF6FF70804503D034F8198019F1ED
S31508000A600109414689B2DFF8080CC05D2844FFF742
S31508000A709EFB1FFA88F8B8F1000F01D14FF6FF78F0
S31508000A807F1C0D2FE3D31FFA88F84FF6FF708045B9
S31508000A9003D034F81900002801D156F040062E700C
S31508000AA0BDE8F18352526141727241617CB504001E
S31508000AB016001D000B222000FFF78CFB062D16D30F
S31508000AC03088002813D03188B61C00201028F7D2A9
S31508000AD089B211F0010212EB450589B24908EA0309
S31508000AE003D585F4883595F02105401CEEE70720E7
S31508000AF015F00F013031C9B23A2900DBC91D6A4623
S31508000B001154401E2D09002DF2D17E216A4611543A
S31508000B10002100E0491C814202D2625C202AF9D1F8
S31508000B200A00511C082803D26B461B5C401C00E0D7
S31508000B302023A3540829F3D373BD00210B220B00ED
S31508000B40DBB2C90111EB530103785918401C521E38
S31508000B50002AF4D10800C0B270472DE9F843040012
S31508000B600E00042527684FF0FF084FF0FF09A0691B
S31508000B7000282ED0A1693800FFF77FFB0500EDB2EB
S31508000B80002D26D1E0690078C0B2002801D10425DD
S31508000B901FE0E169C97A11F03F01A171C0B2E528E9
S31508000BA00DD0C0B22E280AD0C9B231F02002082AC8
S31508000BB001D1012200E00022D2B2B24212D04FF097
S31508000BC0FF0800212000FFF7B8FD0500EDB2002D53
S31508000BD0CDD0EDB2002D01D00020A0612800C0B212
S31508000BE0BDE8F283C9B20F2920D1410607D5E169CC
S31508000BF091F80D9010F0BF00804621696162414668
S31508000C00C0B2C9B288420ED14846E169497BC0B232
S31508000C10884208D1E169A06AFFF7BFFE002802D022
S31508000C20B8F10108CDE74FF0FF08CAE75FFA88F880
S31508000C30B8F1000F06D1E069FFF77FFF5FFA89F97F
S31508000C40814502D05FF0FF306062C2E72DE9F041CE
S31508000C500400256800212000FFF71DFD80465FFA85
S31508000C6088F8B8F1000F02D04046C0B271E0FF27FD
S31508000C703E005FF0FF306062A1692800FFF7FDFAC9
S31508000C8080465FFA88F8B8F1000F60D1E06900780D
S31508000C90C0B2002802D15FF0040858E0E169C97AB9
S31508000CA011F03F01A171C0B2E52804D00A0707D5A3
S31508000CB0C9B20F2904D0FF265FF0FF3060623CE01E
S31508000CC0C9B20F2920D1A16A002936D0410606D516
S31508000CD0E1694F7B10F0BF000600216961623100AF
S31508000CE0C0B2C9B288420DD13800E169497BC0B2A9
S31508000CF0884207D1E169A06AFFF7FCFD002801D008
S31508000D00761E1AE0FF2618E0F6B2002E06D13E003F
S31508000D10E069FFF712FFF6B2864218D0206AC07A59
S31508000D20C00706D40B22216AE069FFF763FA002898
S31508000D300DD0FF265FF0FF30606200212000FFF72C
S31508000D40FCFC80465FFA88F8B8F1000F94D040465C
S31508000D50C0B2BDE8F0812DE9F04784B004002568EB
S31508000D60276AD4F82880F87AA021084201D00620FC
S31508000D709BE05FF0000901E019F1010938F8190054
S31508000D800028F9D10C2239006846FFF723FA9DF8A6
S31508000D900B00C00728D50020F8720020A0625FF07B
S31508000DA0010A01E01AF1010ABAF1640F0CD253469E
S31508000DB0424669463800FFF779FE2000FFF746FFEE
S31508000DC00600F6B2002EEDD0BAF1640F01D1072065
S31508000DD06BE0F6B2042E02D03000C0B265E09DF892
S31508000DE00B00F872C4F828809DF80B00800706D51A
S31508000DF019F10C000D21B0FBF1F0471C00E00127AA
S31508000E0039002000FFF722FD0600F6B2002E2DD18C
S31508000E107F1E002F2AD02069B0EB47112000FFF76C
S31508000E203AFC0600F6B2002E20D1206AFFF785FEAE
S31508000E308046A1692800FFF720FA0600F6B2002EC0
S31508000E4014D14346DBB23A00D2B2E169A06AFFF791
S31508000E50E5FD0120E87000212000FFF76EFC060082
S31508000E60F6B2002E02D17F1E002FE2D1F6B2002E76
S31508000E7019D1A1692800FFF700FA0600F6B2002E7C
S31508000E8011D120220021E069FFF7AEF90B22216A71
S31508000E90E069FFF79FF9206AC07A10F01800E16947
S31508000EA008730120E8703000C0B204B0BDE8F087CE
S31508000EB070B5040025682669606A10F1010F01D132
S31508000EC0002003E0616A2000FFF7E5FBC0B20028B6
S31508000ED019D1A1692800FFF7D0F9C0B200280ED1B0
S31508000EE0E521E26911700121E9702169B14206D252
S31508000EF000212000FFF721FCC0B20028E9D0C0B2CB
S31508000F00042800D10220C0B270BDF8B504000D0057
S31508000F100020A875A06900287BD0606A10F1010F2F
S31508000F201CD00026A76A03E005EB06018875761C27
S31508000F303888BF1C010089B200290BD0002180B275
S31508000F4001F030FD80B2002801D1002602E0FF2E14
S31508000F50EAD30026002005EB060188750020060066
S31508000F6005EB0601897DFFE70B2E31D2E269925D1A
S31508000F70761CD2B2202AF7D0D2B2052A00D1E522B1
S31508000F80092E0BD189B2002903D12E2305EB0007C0
S31508000F90BB752E2305EB00077B72401C05EB00038F
S31508000FA05A7289B2002911D1D2B2B2F141031A2B71
S31508000FB009D2092E01D3102300E00823E7693F7BF5
S31508000FC01F4200D0203205EB00039A75401CCBE780
S31508000FD089B2002908D1002105EB00029175E16963
S31508000FE0097B002900D10020002128444172E069CC
S31508000FF0C07A2872E0691C30FFF7CDF82860E069EE
S315080010001830FFF7C1F8A880E0691630FFF7BCF87A
S31508001010E880F1BD2DE9F84F04008846D8F800901D
S31508001020A06A00900026350003E0009820F81670A4
S31508001030761C19F805706D1CBFB2202F05DBBFB2F0
S315080010402F2F02D0BFB25C2F13D119F805002F2815
S3150800105003D019F805005C2801D16D1CF5E709EBEA
S315080010600500C8F80000BFB2202F20DA5FF0040898
S3150800107021E0FF2E01D3062093E007F0FF070121A8
S31508001080380080B201F08EFC0700BFB2002F01D1F4
S31508001090062086E0BFB2802FC7DABFB23900DFF874
S315080010A02C0CFFF7B6F80028BFD0062079E05FF0D1
S315080010B0000800E0761E002E0AD0009800EB4600D5
S315080010C030F8027CBFB2202FF4D0BFB22E2FF1D059
S315080010D00020009921F81600002E01D1062060E0B4
S315080010E00B222021206AFFF77FF8002500E06D1CFF
S315080010F0009830F815002028F9D0009830F8150027
S315080011002E28F4D0002D03D058F0030800E0761EF0
S31508001110002E06D0009800EB460030F8020C2E2868
S31508001120F5D15FF00009CA465FF0080B01E058F0F8
S315080011300308009830F815706D1CBFB2002F32D125
S31508001140206A0078E52802D10520216A0870BBF1DB
S31508001150080F01D15FEA8A0A5FFA8AFA1AF00C00C8
S315080011600C2805D05FFA8AFA1AF00300032801D181
S3150800117058F002085FEA88700FD45FFA8AFA1AF004
S315080011800300012801D158F010085FFA8AFA1AF00C
S315080011900C00042801D158F00808206A80F80B8052
S315080011A00020BDE8F28FBFB2202FC0D0BFB22E2FCD
S315080011B001D1B542BBD1D94501D2B54213D1BBF154
S315080011C00B0F02D158F00308BAE7B54201D058F020
S315080011D00308AE42B4D335005FF008095FF00B0B85
S315080011E05FEA8A0AA5E7BFB2802F10DB0021380024
S315080011F080B201F0D7FB0700BFB2002F05D0DFF899
S31508001200840CBFB2384410F8807C58F00208BFB28C
S31508001210002F07D0BFB23900DFF86C0CFEF7F9FFD4
S31508001220002803D05F2758F003080FE0BFB2B7F1D4
S3150800123041001A2802D25AF0020A07E0BFB2B7F1F3
S3150800124061001A2802D25AF0010A203F206A00F8E3
S31508001250097019F101096CE773B5040025002E68B9
S3150800126002E00198401C0190019800782F28F8D0D8
S31508001270019800785C28F4D00020A86001980078CE
S31508001280202811D28020216AC87200212000FFF789
S3150800129002FA25E02069C005C00D304410F130017E
S315080012A03000FFF700FBA86001A92000FFF7B2FE97
S315080012B0C0B2002814D12000FFF7C8FC216AC97AF9
S315080012C0C0B2002806D0C0B2042802D1490700D40B
S315080012D0052005E0490703D4A879C006DAD4052015
S315080012E0C0B276BD10B45FF0FF310268002A1BD089
S315080012F0036800E05B1C1A78202A02D31A783A2A77
S31508001300F8D11A783A2A0ED102681478303C521C61
S315080013100A2C06D29A4204D1002C02D121005B1C69
S315080013200360080001E00021080010BC704710B5F2
S3150800133004000020E0705FF0FF30E0622000FEF756
S315080013409CFF002801D0042022E004F22E20FEF79C
S315080013501BFF4AF65521884201D0032018E014F1F4
S315080013606600FEF718FF20F07F40DFF8741B8842FE
S3150800137001D100200CE014F18200FEF70CFF20F0EA
S315080013807F40DFF85C1B884201D1002000E0022084
S3150800139010BDF0B585B00F00150000213960FFF7C4
S315080013A0A1FF0600002E01D50B205EE1DFF8340B05
S315080013B050F82640002C01D10C2056E13C6015F06F
S315080013C0FE05207800280DD0607801F012F9C107D3
S315080013D008D4EDB2002D03D0400701D50A2044E118
S315080013E0002042E1002020706670607801F05EF807
S315080013F0C10701D5032038E1EDB2002D03D040071F
S3150800140001D50A2031E1002529002000FFF78FFFCA
S315080014100600F6B2022E2AD1002704E0002069460B
S3150800142041F827007F1C042F0BD2380120444FF4C3
S31508001430F771084401790029F0D00830FEF7ABFEB1
S31508001440EDE70027002F00D07F1E684650F827508A
S31508001450002D05D029002000FFF769FF060000E0EF
S315080014600326F6B2022E02DB7F1C042FEDD3F6B25A
S31508001470042E01D10120F8E0F6B2022E01DB0D2080
S31508001480F3E014F13B00FEF77FFEB0F5007F01D0D4
S315080014900D20EAE014F14600FEF776FE0700002F5D
S315080014A004D114F15400FEF776FE0700A76194F8FC
S315080014B04000A070A078012804D0A078022801D0A6
S315080014C00D20D2E0A078474394F83D0060816089FA
S315080014D0002804D060896189491E084201D00D2080
S315080014E0C3E014F14100FEF74FFE2081207A0F2158
S315080014F0084201D00D20B8E014F14300FEF744FE7F
S315080015000600002E04D114F15000FEF744FE060032
S3150800151014F13E00FEF738FE80B2002801D10D20F6
S31508001520A3E017FA80F1228911EB12118E4201D23B
S315080015300D209AE0721A6389B2FBF3F2002A01D1F0
S315080015400D2092E0012640F6F6739A4200D3022651
S315080015504FF6F6739A4200D30326921C6261E56140
S3150800156015FA80F020624819A062F6B2032E14D14B
S3150800157014F15A00FEF708FE002801D00D2074E089
S315080015802089002801D00D206FE014F15C00FEF7D9
S3150800159002FE60626069800015E02089002801D19A
S315080015A00D2062E0206A38186062F6B2022E02D177
S315080015B06069400007E0606903214843217D11F016
S315080015C0010111EB5000A16900F2FF10B1EB502F99
S315080015D001D20D2049E05FF0FF3020612069E0600C
S315080015E080202071F6B2032E32D114F16000FEF786
S315080015F0CBFD01282CD1691C2000FEF73EFE0028F1
S3150800160026D10020207104F22E20FEF7BDFD4AF6F1
S31508001610552188421CD114F13000FEF7BCFDDFF8D5
S315080016209419884214D14FF405702044FEF7B3FD8F
S31508001630DFF8841988420BD14FF406702044FEF770
S31508001640AAFD20614FF407702044FEF7A4FDE06070
S315080016502670DFF868090088401CDFF860190880E2
S31508001660DFF858090088E080002005B0F0BD0000CA
S31508001670D87A000838B505000C00002D11D0286866
S3150800168000280ED02868007800280AD02868C08864
S31508001690A988884205D12868407800F0AAFFC007C3
S315080016A003D500202060092002E028682060002079
S315080016B0C0B232BD13B582B01400039800906846D4
S315080016C0FFF710FE002801D50B2020E0DFF81418DC
S315080016D051F82010002901D000220A700299002929
S315080016E002D00021029A11700299DFF8F82742F811
S315080016F020100298002802D0E4B2012C01D0002064
S3150800170005E0002202A903A8FFF743FEC0B204B011
S3150800171010BD2DE9F2418FB004001500002C01D14F
S315080017200920B0E00020206015F01F052A00D2B27B
S3150800173069460FA8FFF72DFE0600F6B2002E40F008
S31508001740A080009801900CA80990DFF874080B9007
S315080017500F9901A8FFF780FD0600F6B2002E04D106
S315080017600998C07A000600D506261C20054253D0E3
S31508001770F6B2002E09D0F6B2042E03D101A8FFF75F
S31508001780EAFA060055F0080509E09DF80A00112155
S31508001790084201D0072602E0680700D50826F6B2F7
S315080017A0002E49D1280747D5DFF8188841460898FA
S315080017B00E30FEF703FD414608981630FEF7FEFC8C
S315080017C020200899C87208990098FFF76CF8070056
S315080017D0002208990098FFF779F8002108981C302C
S315080017E0FEF7ECFC01200099C870002F24D0009861
S315080017F0D0F82C800022390001A8FEF7A2FE0600C8
S31508001800F6B2002E18D141460098FEF736FD0600BE
S31508001810781E0099C8600FE0F6B2002E0CD19DF82C
S315080018200A00C00601D5042606E0A80704D59DF8D7
S315080018300A00C00700D50726F6B2002E08D12807E9
S3150800184001D555F020050098C06A206208986062A4
S31508001850F6B2002E15D108990098FFF724F8A06073
S3150800186008981C30FEF797FCE060002060740020A2
S3150800187060610020E0612574009820600098C088A7
S31508001880A0803000C0B210B0BDE8F0812DE9F04765
S3150800189082B0050016001F000C000020386069465B
S315080018A02800FFF7E7FEC0B2002804D1687C0100D3
S315080018B0C9B2002901D0C0B2BDE0287CC00701D456
S315080018C00720B8E0E8686969401AB04220D20600E5
S315080018D01EE0C5F81C906869C005C00DD0F50078F3
S315080018E0464500D2B04642466869C005C00D284440
S315080018F010F128012000FEF76DFC4444686918EBD6
S3150800190000006861386818EB00003860B6EB080616
S31508001910002E00F08F806869C005DCD168690099DF
S315080019204989491E11EA5028B8F1000F16D168698D
S31508001930002801D1A86803E0A9692800FEF713FD6D
S31508001940022803D202206874022074E010F1010F05
S3150800195003D10120687401206DE0A861A969009887
S31508001960FEF7F5FC8146B9F1000F03D10220687431
S31508001970022060E018EB09095FEA562ABAF1000F5F
S3150800198030D0009840891AEB0801884203D20098A3
S315080019904089B0EB080A53464A4621000098407829
S315080019A000F030FE002803D001206874012042E0D0
S315080019B0287C400611D5E869B0EB090050450CD2E1
S315080019C04FF4007215F12801E869B0EB09004FF4ED
S315080019D0007358432044FEF7FDFB4FF4007000FBEC
S315080019E00AF88AE7E86948453FF473AF287C400659
S315080019F011D50123EA6915F128010098407800F00D
S31508001A004AFE002803D001206874012013E0287CD0
S31508001A1010F0BF00287401234A4615F128010098E2
S31508001A20407800F0EFFD00283FF453AF01206874BA
S31508001A30012000E00020BDE8F6872DE9F04782B0D6
S31508001A40050017001E000C000020306069462800BB
S31508001A50FFF710FEC0B2002804D1687C0100C9B2A5
S31508001A60002901D0C0B23BE0287C800701D40720BA
S31508001A7036E068693818696988420CD25FF0FF3029
S31508001A806969471A07E0E868E860306818EB0000FB
S31508001A903060B7EB0807002F1DD06869C00540F015
S31508001AA0A580686900994989491E11EA5028B8F144
S31508001AB0000F29D16869002807D1A868002808D12D
S31508001AC000212800FEF781FD03E0A9692800FEF73A
S31508001AD07CFD002806D1287C50F0200028740020C0
S31508001AE0BDE8F687012803D1022068740220F7E7CB
S31508001AF010F1010F03D1012068740120F0E7A861F5
S31508001B00A968002900D1A860287C400611D50123C0
S31508001B10EA6915F128010098407800F0BCFD002814
S31508001B2003D0012068740120DAE7287C10F0BF0092
S31508001B302874A9690098FEF70AFC8146B9F1000FD6
S31508001B4003D1022068740220CAE718EB09095FEA84
S31508001B50572ABAF1000F32D0009840891AEB0801CB
S31508001B60884203D200984089B0EB080A53464A4691
S31508001B7021000098407800F08EFD002803D001204F
S31508001B8068740120ACE7E869B0EB0900504511D24A
S31508001B904FF40072E869B0EB09004FF4007148434E
S31508001BA004EB000115F12800FEF714FB287C10F061
S31508001BB0BF0028744FF4007000FB0AF82BE0E869B0
S31508001BC0484511D06869E96888420DD201234A461A
S31508001BD015F128010098407800F014FD002803D07C
S31508001BE00120687401207BE7C5F81C906869C00568
S31508001BF0C00DD0F50078474500D2B84642462100C8
S31508001C006869C005C00D28442830FEF7E3FA287C29
S31508001C1050F0400028744444686918EB0000686175
S31508001C20E86869698842BFF42EAF68692CE770B521
S31508001C3082B0040069462000FFF71CFDC0B20028E8
S31508001C4041D1217C89063ED5207C40060FD501234B
S31508001C50E26914F128010098407800F01CFD00287C
S31508001C6001D0012030E0207C10F0BF002074DFF89E
S31508001C705453216A0098FEF700FBC0B2002822D10F
S31508001C80666AF07A50F02000F072A2683100206887
S31508001C90FEF71CFEE16816F11C00FEF78FFA290014
S31508001CA016F11600FEF78AFA002116F11200FEF761
S31508001CB07EFA01200099C8700098FEF7FCFA217C8C
S31508001CC011F0DF012174C0B276BD0000387B000830
S31508001CD010B582B004002000FFF7A9FFC0B20028A3
S31508001CE008D169462000FFF7C5FCC0B2002801D11B
S31508001CF000212160C0B216BD2DE9F04182B0040072
S31508001D000D0069462000FFF7B5FC0600F6B2002E66
S31508001D1004D1667C3000C0B2002802D03000C0B2C0
S31508001D20ADE0E068A84203D2207C800700D4E568CD
S31508001D30606900276761002D6BD0009949894FF4C7
S31508001D40007202FB01F8002810D0411EB1FBF8F121
S31508001D506A1EB2FBF8F28A4208D3401EB8F10101A6
S31508001D608843606160692D1AA06915E0A06800289B
S31508001D7011D100212000FEF728FC012803D10220FA
S31508001D80607402207BE010F1010F03D1012060741A
S31508001D90012074E0A060A061002807D139E0A061A5
S31508001DA0616918EB01016161B5EB0805A84509D21F
S31508001DB0217C890716D501002000FEF706FC0028BD
S31508001DC014D14546616969186161E90521D00100A8
S31508001DD00098FEF7BCFA0700002F18D1022060749D
S31508001DE002204CE001002000FEF7BDFA10F1010FB9
S31508001DF003D101206074012041E0022803D3009931
S31508001E0049698842CBD302206074022037E017EB79
S31508001E1055276069C00526D0E069874223D0207C13
S31508001E20400611D50123E26914F12801009840788B
S31508001E3000F031FC002803D00120607401201EE068
S31508001E40207C10F0BF00207401233A0014F1280109
S31508001E500098407800F0D6FB002803D00120607473
S31508001E6001200CE0E761E0686169884205D2606993
S31508001E70E060207C50F0200020743000C0B2BDE83D
S31508001E80F6810000B87400085C7B000831B58EB096
S31508001E900C00002203A90EA8FFF77BFA0500EDB295
S31508001EA0002D18D168460B90DFF814010D900E9995
S31508001EB003A8FFF7D1F90500EDB2002D0BD10B9859
S31508001EC0C07A000601D5062505E0002C03D02100BE
S31508001ED003A8FFF71AF82800C0B20FB030BD0000FB
S31508001EE0464154007820002031B59AB000240222D9
S31508001EF069461AA8FFF74DFA050000980190EDB259
S31508001F00002D53D10CA809902D480B901A9901A8B9
S31508001F10FFF7A2F90500EDB2002D47D10998C07A5E
S31508001F20000601D5062504E09DF80A00C00700D57D
S31508001F300725EDB2002D20D108990098FEF7B3FCCD
S31508001F4004009DF80A00C00617D500980F90119452
S31508001F5000210FA8FEF79FFB0500EDB2002D0CD15E
S31508001F6000210FA8FEF7F9FD0500EDB2002D00D1FE
S31508001F700725EDB2042D00D10025EDB2002D15D1AF
S31508001F8001A8FEF795FF0500EDB2002D07D1002C3C
S31508001F9005D00022210001A8FEF7D3FA0500EDB20C
S31508001FA0002D03D10098FEF786F905002800C0B277
S31508001FB01BB030BD5252614172724161A4200020AB
S31508001FC060190020000061482DE9FC4104000F005B
S31508001FD0904600262500FFE7781E864213DA6B46F0
S31508001FE0012201A94046FFF751FC009801280AD1B1
S31508001FF09DF80400C0B20D28EED028706D1C761C22
S31508002000C0B20A28E8D100202870002E00D100248A
S315080020102000BDE8F68170B582B004000D00EDB26F
S315080020200A2D03D10D212000FFF7F5FF6668002E63
S3150800203017D404EB06000573761C3D2E0DDB6B46A4
S31508002040320014F10C012068FFF7F7FC0098B04243
S3150800205001D1002601E05FF0FF366660A068401CEB
S31508002060A06073BD10B594B00400019100200290E1
S315080020700298039004E0217801A8FFF7CCFF641CBE
S3150800208020780028F7D1029800280DD46B46029ACA
S3150800209004A90198FFF7D1FC002805D102980099F8
S315080020A0884201D1039801E05FF0FF3014B010BDFB
S315080020B01CB54FF48051DFF8DC0800F054FD02200F
S315080020C08DF8050001208DF8040000208DF8070022
S315080020D000208DF806004FF4004000906946DFF8AE
S315080020E0B40800F0E3FC4FF40041DFF8A80800F05C
S315080020F03AFD002413E00221DFF89C0800F09FFD5A
S315080021000028F8D0FF21DFF8900800F088FD0121AB
S31508002110DFF8840800F093FD0028F8D0641C0A2C28
S31508002120E9D34FF40040009002208DF80400022005
S315080021308DF8050000208DF8060002208DF80700AE
S315080021406946DFF8500800F0B1FC13BD00B587B04A
S315080021500121022000F0EAFD01214FF4804000F041
S3150800216005FE4FF48050009002208DF805000120EE
S315080021708DF8040000208DF8070000208DF8060071
S315080021806946DFF8100800F091FC4FF48051DFF83B
S31508002190040800F0E8FC05220D21DFF8F80700F036
S315080021A0E6FC05220E21DFF8EC0700F0E0FC05222C
S315080021B00F21DFF8E00700F0DAFC4FF460400090EA
S315080021C002208DF8040002208DF8050000208DF805
S315080021D0060002208DF807006946DFF8B80700F008
S315080021E065FC0020ADF808004FF48270ADF80A00CF
S315080021F00020ADF80C000020ADF80E000020ADF868
S3150800220010004FF40070ADF812003020ADF814003D
S315080022100020ADF816000720ADF8180002A9DFF86F
S31508002220780700F0CDFC0021DFF86C0700F0F9FC18
S315080022300121DFF8640700F0E2FCFFF739FF07B079
S3150800224000BD00B585B00021DFF84C0700F0D7FCCB
S315080022500020ADF800004FF48270ADF802000020AF
S31508002260ADF804000020ADF806000020ADF808001F
S315080022704FF40070ADF80A000020ADF80C000020FD
S31508002280ADF80E000720ADF810006946DFF808071C
S3150800229000F096FC0021DFF8000700F0C2FC0121DF
S315080022A0DFF8F40600F0ABFC05B000BDDFF8EC067D
S315080022B0007850F00100DFF8E4160870704780B522
S315080022C0C0B2010089B2DFF8D00600F0A8FC0121EF
S315080022D0DFF8C40600F0B3FC0028F8D0DFF8B8062B
S315080022E000F09BFCC0B202BD10B50400FF20FFF74A
S315080022F0E6FF207010BD38B500F09AFD10F5FA75A6
S31508002300FF20FFF7DCFF0400E4B2FF2C03D000F047
S315080023108FFDA842F4D3E4B2FF2C01D1012000E0DE
S31508002320002032BD80B54FF48051DFF8680600F012
S315080023301AFCFF20FFF7C3FF01BD80B54FF480519B
S31508002340DFF8500600F011FCFF20FFF7B8FFFFF793
S31508002350D2FF002801D0012002E0FFF7E3FF0020AA
S3150800236002BDF8B504000D0000F062FD10F1640727
S31508002370FF20FFF7A4FF0600F6B2FF2E03D100F0F8
S3150800238057FDB842F4D3F6B2FE2E01D0002011E074
S315080023902000FFF7A9FF641C2000FFF7A5FF641CB7
S315080023A0AD1E002DF4D1FF20FFF789FFFF20FFF7B0
S315080023B086FF0120F2BD38B504000D00FFF79BFF2C
S315080023C0002801D1002024E02800C0B2FFF777FFDB
S315080023D0EDB2FD2D1CD04FF400752078FFF76FFF86
S315080023E0641C2078FFF76BFF641CAD1E002DF4D12A
S315080023F0FF20FFF764FFFF20FFF761FFFF20FFF7CD
S315080024005EFFC0B210F01F00052801D0002000E0D2
S31508002410012032BD38B504000D0020060AD514F097
S315080024207F0400213720FFF7F5FFC0B2022801DB41
S31508002430C0B23AE0FFF776FFFFF77FFF002801D129
S31508002440FF2032E054F04000C0B2FFF738FF280EF4
S31508002450C0B2FFF734FF280CC0B2FFF730FF280AD6
S31508002460C0B2FFF72CFF2800C0B2FFF728FF0125EE
S31508002470E4B2002C00D19525E4B2082C00D18725BA
S315080024802800C0B2FFF71BFFE4B20C2C02D1FF20D4
S31508002490FFF715FF0A25FF20FFF711FF010603D5F1
S315080024A06D1EEDB2002DF6D1C0B232BD70B582B048
S315080024B0C0B2002801D001209AE0DFF8E0040078D5
S315080024C0800703D5DFF8D404007891E0FFF73EFED5
S315080024D04FF48051DFF8BC0400F047FB00250021CB
S315080024E00020FFF797FF012869D100F0A1FC10F53D
S315080024F07A764FF4D5710820FFF78CFF01283CD176
S31508002500002406E0FF20FFF7DAFE6946E4B2085524
S31508002510641CE4B2042CF5DB9DF8020001284ED1B8
S315080025209DF80300AA284AD100F082FCB04206D2E0
S315080025305FF08041A920FFF76DFF0028F4D100F075
S3150800254077FCB0423BD200213A20FFF763FF002810
S3150800255035D1002406E0FF20FFF7B1FE6946E4B254
S315080025600855641CE4B2042CF5DB9DF8000040060F
S3150800257001D50C2523E0042521E00021A920FFF739
S3150800258049FF022802DA0225A92401E001250124CF
S3150800259000F04EFCB04206D200212000C0B2FFF780
S315080025A039FF0028F4D100F043FCB04206D24FF4BC
S315080025B000711020FFF72EFF002800D00025EDB28D
S315080025C0DFF8DC030560FFF7ADFEEDB2002D0AD09B
S315080025D0DFF8C803007810F0FE00DFF8C0130870B3
S315080025E0FFF72FFE01E0FFF761FEDFF8B003007882
S315080025F076BDC0B2002801D0012002E0DFF89C03B6
S315080026000078704738B50C0011001D00C0B20028CC
S3150800261001D1002D01D104203CE0DFF880030078C9
S31508002620C00701D5032035E0DFF8740300780007FA
S3150800263002D44FF400704143012D0DD11120FFF74C
S31508002640E9FE00281ED14FF400712000FFF789FE2D
S31508002650002817D0002515E01220FFF7DBFE00281A
S3150800266010D14FF400712000FFF77BFE002805D03B
S315080026704FF4007004446D1E002DF2D100210C2089
S31508002680FFF7C8FEFFF74EFE002D01D0012000E03F
S315080026900020C0B232BD70B50C0015001E00C0B2D5
S315080026A0002801D1002E01D104204CE0BB48007857
S315080026B0C00701D5032046E0B8480078400701D591
S315080026C0022040E0B6480078000702D44FF40070B4
S315080026D04543012E0DD129001820FFF79BFE00283F
S315080026E029D1FE212000FFF766FE002823D0002608
S315080026F021E0AB48007810F0060F03D03100972090
S31508002700FFF788FE29001920FFF784FE002812D15A
S31508002710FC212000FFF74FFE002805D04FF400707B
S315080027200444761E002EF3D1FD210020FFF743FE58
S31508002730002800D10126FFF7F5FD002E01D0012063
S3150800274000E00020C0B270BD30B585B0140022008C
S31508002750C0B2002801D004201AE190480078C007CA
S3150800276001D5032014E10125C9B2002913D0012996
S3150800277017D003295FD00A2900F0BC800B2900F086
S31508002780BE800C2900F0C9800D2900F0D4800E29DE
S3150800279000F0E480F7E0FFF7D0FD002800D0002520
S315080027A0F2E000210920FFF735FE002842D110216A
S315080027B06846FFF7D6FD00283CD09DF80000C0B259
S315080027C08009C0B2012810D19DF809009DF80810AB
S315080027D0090251FA80F09DF8071011F03F0110EB3D
S315080027E00140401C8002206023E09DF8050010F09F
S315080027F00F009DF80A10C9B210EBD1109DF8091008
S31508002800490011F006010818851C9DF80800C0B299
S3150800281080099DF80710890051FA80F09DF8061086
S3150800282011F0030110EB8120401CB5F10901884025
S3150800283020600025A8E05A480078400720D50021E6
S315080028408D20FFF7E7FD002853D1FF20FFF737FD5E
S3150800285010216846FFF785FD00284AD0302503E099
S31508002860FF20FFF72CFD6D1EEDB2002DF8D11020CC
S315080028709DF80A10C9B2090988402060002538E089
S3150800288000210920FFF7C6FD002832D1102168462D
S31508002890FFF767FD00282CD041480078800713D53C
S315080028A09DF80A00400010F07E009DF80B10C9B292
S315080028B0C90950FA81F0401C9DF80D10C9B2890962
S315080028C0491E8840206013E09DF80A00C0F3840082
S315080028D0C0B2401C9DF80B10C90011F018019DF8F4
S315080028E00B20D2B2520951FA82F1491C48432060A2
S315080028F0002549E02A4800681070002544E00021B8
S315080029000920FFF787FD002806D110212000FFF7D0
S3150800291028FD002800D0002536E000210A20FFF710
S3150800292079FD002806D110212000FFF71AFD00289E
S3150800293000D0002528E000213A20FFF76BFD00288B
S315080029400BD1002505E0FF20FFF7B9FCEDB2605575
S315080029506D1CEDB2042DF6DB002515E01048007855
S3150800296040070FD500218D20FFF754FD002809D117
S31508002970FF20FFF7A4FC40212000FFF7F2FC002807
S3150800298000D0002500E00425FFF7CCFC2800C0B2E3
S3150800299005B030BD0004024000380040DD000020CC
S315080029A08020002080B2802801DA010020E000297A
S315080029B00CD080B2FF2801DD002119E0384980B229
S315080029C001EB4000B0F58070018811E0002100E0BD
S315080029D0491C89B2802907DA0200314B89B233F8DB
S315080029E0113092B29A42F3D111F1800000F0FF0142
S315080029F0080080B2704730B480B2B0F5805F01DA63
S31508002A00284A07E0284A05E089B2002902D1A4B27B
S31508002A1002EB44021388921C9BB2002B05D00100DE
S31508002A201C0089B2A4B2A14200D235E01488921CD7
S31508002A30210089B2090A04F0FF0480B2A4B214FA8C
S31508002A4083F5A842E0DA89B200290CD0022915D00C
S31508002A500FD3042916D013D3062917D014D308295F
S31508002A6018D015D318E080B29BB2C01A32F81000FD
S31508002A7012E0C11A11F00101401A0DE010380BE0FE
S31508002A80203809E0303807E01A3805E0083003E056
S31508002A90503801E0B0F5E35080B230BC7047000012
S31508002AA0FC720008F86D0008FC73000830B40022B8
S31508002AB000230024002247E0012393400C681C40B1
S31508002AC09C4240D1036803241500EDB26D00AC406A
S31508002AD0A343036003680C791500EDB26D00AC40A2
S31508002AE0234303600B79012B02D00B79022B1AD1F1
S31508002AF0836803241500EDB26D00AC40A3438360E0
S31508002B0083684C791500EDB26D00AC4023438360B1
S31508002B10436801249440A343436043688C799440F6
S31508002B20A4B223434360C36803241500EDB26D00C5
S31508002B30AC40A343C360C368CC791500EDB26D0001
S31508002B40AC402343C360521C102AB5D330BC70472F
S31508002B500022006989B2084201D0012200E0002261
S31508002B601000C0B27047018370474183704770B444
S31508002B7000230023D2B211F00703DBB29B0012FA3E
S31508002B8003F389B2CA1000EB820289B2CC1000EBBB
S31508002B908404246A0F2511F00706F6B2B600B5407C
S31508002BA0AC43146289B2CA1000EB8202126A13435C
S31508002BB089B2C91000EB8100036270BC704700003F
S31508002BC010B40022028812F441520B884C88234321
S31508002BD08C882343CC8823430C8923434C8923437D
S31508002BE08C892343CC8923431A430280828B4FF274
S31508002BF0FF731A408283098A018210BC7047C9B2E2
S31508002C00002904D0018851F04001018004E00188C0
S31508002C104FF6BF72114001807047808970478181E5
S31508002C207047C9B2002904D0018851F400510180C7
S31508002C3004E001884DF6FF721140018070470022BA
S31508002C400089084201D0012200E000221000C0B22B
S31508002C5070470000002100210021022200210222E3
S31508002C60DFF86811096811F00C01002904D004295D
S31508002C7006D0082908D033E0DFF85811016032E0A1
S31508002C80DFF8541101602EE0DFF844110968C1F33A
S31508002C908051DFF83C21126812F03F0200290AD061
S31508002CA0DFF83411B1FBF2F1DFF824211268C2F320
S31508002CB08812514309E0DFF81C11B1FBF2F1DFF885
S31508002CC010211268C2F388125143DFF804211268F2
S31508002CD0C2F30142521C5200B1FBF2F1016002E05C
S31508002CE0DFF8F0100160DFF8E410096811F0F00170
S31508002CF00909DFF8E820515C0268CA404260334996
S31508002D00096811F4E051890ADFF8D020515C42685D
S31508002D10CA4082602D49096811F46041490BDFF801
S31508002D20BC20515C4268CA40C2607047C9B20029DB
S31508002D3005D02B49096808432949086005E0284950
S31508002D40096831EA0000264908607047C9B20029B7
S31508002D5005D02449096808432249086005E0214945
S31508002D60096831EA00001F4908607047C9B200299E
S31508002D7005D01D49096808431B49086005E01A493A
S31508002D80096831EA0000184908607047C9B2002985
S31508002D9005D01649096808431449086005E013492F
S31508002DA0096831EA0000114908607047C9B200296C
S31508002DB005D00F49096808430D49086005E00C4924
S31508002DC0096831EA00000A49086070470838024075
S31508002DD0043802400024F40000127A0000000020A3
S31508002DE03038024034380240403802404438024005
S31508002DF02038024080B500F00DF8104810490860E8
S31508002E0000201049086005200F49086000200F4976
S31508002E10086001BD00200C49086070470A48006830
S31508002E20C00304D509480068401C08490860704773
S31508002E3080B5FFF7F3FF0548006802BD3F90020022
S31508002E4014E000E018E000E010E000E08420002034
S31508002E5000215FF0FF32C3685A607FF08042C36882
S31508002E605A6151F0004151F40061C06881617047B0
S31508002E7070B582B0040000250026002000900320CB
S31508002E8000F054FDE06800690090761CB848864258
S31508002E9001D300201AE00098C00F0028EFD00026C2
S31508002EA0009850F0010000900098E1680861E06819
S31508002EB000690090761CAE48864202D20098C00788
S31508002EC0F5D4032000F032FD2800C0B276BD70B4F8
S31508002ED004000020E578002D13D1002500269BB2BA
S31508002EE0DB1C042593FBF5F5D2B204EB8202D2F87B
S31508002EF0D020002603E00B681360761C091DAE423D
S31508002F00F9D3C0B270BC704710B4002392B2D21C79
S31508002F10042392FBF3F2D0F8D000002303E0046800
S31508002F200C605B1C091D9342F9D3080010BC70475E
S31508002F3030B40A00002300210024C47001248470E0
S31508002F4040248480D2B2012A0DD15FF0A043012229
S31508002F50C27208220270042242704FF4A072C28024
S31508002F60022202720CE0D2B2002A09D1814B002259
S31508002F70C2720C220270062242704FF4A062C2800E
S31508002F80C36013F50062026100220EE013EB4214DF
S31508002F9014F5106400EB8205AC6113EB421414F5CA
S31508002FA0306400EB82056C65521C4478A242EDD36E
S31508002FB013F58062426113F58862C0F8CC200022BE
S31508002FC008E013EB421414F5A06400EB8205C5F87B
S31508002FD09040521C0478A242F3D300220AE04FF430
S31508002FE0805404FB023414F5805400EB8205C5F8BE
S31508002FF0D040521C0478A242F1D313F56062C0F89F
S315080030000C210800C0B230BC704770B5040000251A
S31508003010002000200026207A012825D1E068806B50
S3150800302030F48030617A002901D050F48010E168CC
S3150800303088630020E068C06830F0400030F4800003
S3150800304030F4003030F40020E168C8602000FFF753
S315080030500FFFE078012821D1052060F3440656F0D9
S315080030602006E068866019E0E068C06850F0400015
S31508003070E168C8602000FFF7FBFE002050F48030AE
S3150800308050F4802050F40020617A002901D050F4D1
S315080030908010E1688863142000F053FCE07801286A
S315080030A008D1E0688668052060F3440656F02006D5
S315080030B0E06886602800C0B270BD0021002252F088
S315080030C00102C3689B681A43C06882600800C0B2E0
S315080030D070470021002252F00102C3689B6833EA58
S315080030E00202C06882600800C0B2704710B582B09C
S315080030F00024002200230093009B53F02003009332
S31508003100009B61F38A1300930099C3681961C1682B
S3150800311009690091521C16498A4204D20099C1F3E2
S3150800312040110029F3D1032000F000FC2000C0B2B2
S3150800313016BD10B582B00024002100220092009A24
S3150800314052F010020092009AC3681A61C2681269A6
S315080031500092491C064A914204D2009AC2F3001210
S31508003160002AF3D1032000F0E1FB2000C0B216BD0F
S31508003170410D03000000044010B50024C268D2685F
S3150800318032F0005232F08042C9B2012902D152F01F
S31508003190005204E0C9B2002901D152F08042C06849
S315080031A0C260322000F0CDFB2000C0B210BDC0685E
S315080031B0406910F00100704780B5FFF7F8FF012855
S315080031C001D0012000E00020C0B202BD0021C16884
S315080031D04969C06880690140080070470269126839
S315080031E0C9B261F30102006902607047F8B50400CC
S315080031F00025002100200026002700200020D4F802
S315080032000C1108602069006830F4C0502169086014
S31508003210E07A01282AD103212000FFF7DFFF80206A
S31508003220E1684862202060F31F46802060F30F069D
S31508003230E068866216EB164060F30F07802060F39D
S315080032401F47E068C0F8047117EB1740C0EA070784
S31508003250202060F31F47E068C0F8087117EB174095
S31508003260C0EA0707BFB2E068C0F80C711021200059
S31508003270FFF73CFF2000FFF75CFF0020216908618B
S315080032800020216948615FF0FF30216988610020CC
S315080032902169C86100200FE0002104EB80029269D1
S315080032A0116004EB8001896900220A6104EB800140
S315080032B08969FF228A60401C617888420CD204EB37
S315080032C0800189690968C90F0029E5D0002151F0F4
S315080032D0804151F00061E0E700200FE0002104EB97
S315080032E08002526D116004EB8001496D00220A616B
S315080032F004EB8001496DFF228A60401C6178884290
S315080033000CD204EB8001496D0968C90F0029E5D084
S31508003310002151F0804151F00061E0E7002050F4AF
S315080033208070216909698143084321690861E07849
S3150800333001280ED1002050F0010050F00200402173
S3150800334061F38A0050F48030402161F359402169C5
S315080033500863200000F003F82800C0B2F2BD70B57B
S315080033600400002500260020E16888617FF080407F
S31508003370E16848612000FFF76BFDE078002801D17D
S3150800338056F0100656F4006656F4805656F4005663
S3150800339056F4802656F4002656F0080656F480168B
S315080033A056F4001656F0804656F00406E068806922
S315080033B0B0433043E16888612800C0B270BD00217F
S315080033C000698068400810F00300002805D002282C
S315080033D007D004D3032802D004E0032102E0022127
S315080033E000E001210800C0B2704710B40021002493
S315080033F00269926883691B68520812F00302002A60
S3150800340004D0022A05D001D3032A05D1DB0ADB0240
S3150800341002E0032262F30A038269136054F480749B
S3150800342002695268A2432243006942600800C0B29A
S3150800343010BC704770B40A00002100250023547898
S31508003440012C0AD1147800EB8404A469012592F9A9
S315080034500060B54065F30F0309E0147800EB8404B7
S31508003460646D012592F90060B54065F31F43256830
S31508003470C5F3C036002E0DD1966866F30A05D678D0
S3150800348066F39345D28862F3995555F0805555F4FD
S31508003490004525600269D2691A430069C2610800BD
S315080034A0C0B270BC704770B40A0000210023002423
S315080034B05578012D0BD1157800EB8505AD690126E8
S315080034C092F9002016FA02F262F30F040AE0157860
S315080034D000EB85056D6D012692F9002016FA02F2B9
S315080034E062F31F4433F400432B600269D269A24396
S315080034F00069C2610800C0B270BC704770B500248C
S315080035000023002200234A78012A61D10A7800EBB9
S315080035108202926912680B7800EB83039B691B6928
S315080035204D69002D05D1DB0CDB04012565F3DC4371
S3150800353011E04D6965F312034D698E6875196D1EA4
S315080035408E68B5FBF6F565F3DC43CD78012D02D11F
S31508003550012565F35E730D7800EB8505AD692B6172
S31508003560C378012B06D10B7800EB83039B690D69A1
S315080035705D610EE0CB78012B0BD04B69002B08D090
S31508003580012391F90050AB4005696D6B2B43056922
S315080035906B63CB78012B08D103699B68DB0502D4E2
S315080035A052F0005201E052F0805252F0806252F01E
S315080035B000420B7800EB83039B691A60CA78012ADC
S315080035C04BD14B699BB20A78C968FFF780FC44E087
S315080035D00A7800EB8202526D12680B7800EB8303BF
S315080035E05B6D1B694D69002D06D18D6865F3120365
S315080035F0012565F3DC430EE04D698E6875196D1E6D
S315080036008E68B5FBF6F565F3DC43C3F3C9458E68EA
S31508003610754365F312030D7800EB85056D6D2B6117
S31508003620C378012B05D10B7800EB83035B6D0D691D
S315080036305D61CB78012B07D14B79002B02D052F074
S31508003640005201E052F0805252F0806252F000427D
S31508003650097800EB8100406D02602000C0B270BDA1
S31508003660FCB4002200240023002300934B78012B8E
S3150800367048D185692B682E6900964E69002E09D1B6
S31508003680009EF609F60100960126009F66F3D447C8
S31508003690009715E08E684F69BE4207D28E684E6164
S315080036A08E68009F66F30607009704E04E69009F40
S315080036B066F3060700970126009F66F3D44700972E
S315080036C0009E2E61C678012E05D10E7800EB86067F
S315080036D0B6690F69776153F0806353F000432B6036
S315080036E0C378002B4BD14B69002B48D0012391F9A5
S315080036F0001013FA01F10C430169496B2143006973
S3150800370041633CE00B7800EB83035B6D1B680C7828
S3150800371000EB8404646D246900944C69002C0AD17A
S315080037208C68009D64F3060500950124009D64F3EA
S31508003730D44500950BE08C684C618C68009D64F359
S31508003740060500950124009D64F3D44500950C7880
S3150800375000EB8404646D009D2561C478012C05D1B5
S315080037600C7800EB8404646D0D69656153F0806321
S3150800377053F00043097800EB8100406D03601000A8
S31508003780C0B2F6BC7047002200234B78012B0DD13E
S31508003790097800EB810080690368D90F002901D0F8
S315080037A053F0804353F40013036007E0097800EBF5
S315080037B08100406D036853F4001303601000C0B223
S315080037C0704710B4002200234B78012B04D10B78E4
S315080037D000EB8300806903E00B7800EB8300406D03
S315080037E0036833F40013CC78032C02D0C978022975
S315080037F001D153F0805303601000C0B210BC70476B
S31508003800016989690069C0690140080C7047C9B235
S3150800381000EB8101496D896800694069014008002B
S315080038207047016989690069C069014088B27047B3
S3150800383082B000210091009951F040410091012188
S31508003840009A61F3D44200921821009A61F30602A5
S3150800385000920099426D1161C17801290CD10021AD
S3150800386000F2CC51426D5161416D096851F0004139
S315080038705FF08021406D016002B0704700B583B0EB
S3150800388001210120FFF752FA4FF4C050009003209F
S315080038908DF8050002208DF8040000208DF806003A
S315080038A000208DF8070069461C48FFF7FFF80A2232
S315080038B00B211A48FFF75BF90A220C211748FFF774
S315080038C056F901210420FFF731FA4FF40060009001
S315080038D001208DF8040000208DF8060001208DF8DF
S315080038E0070003208DF8050069460D48FFF7DEF846
S315080038F00C48006830F400600A49086001214FF45A
S315080039008040FFF743FA01218020FFF71FFA0121C3
S315080039105FF08050FFF74AFA07BD0000000002403A
S315080039200008024014080240704700000100481EC3
S31508003930002905D000211C29F8D200BF491CFAE746
S31508003940704780B54FF47A714843FFF7EFFF01BD22
S3150800395080B50020DFF850170870002218A1DFF89C
S315080039604C07FDF7A7FEC0B2002804D07721DFF880
S31508003970400700F02EFC01BDDFF82C070078002870
S3150800398001D1012000E00020704780B500F0B0FCAE
S31508003990012801D1002011E0DFF80C070078002883
S315080039A001D000200AE000F0EEFC012805D1012034
S315080039B0DFF8F4160870012000E0002002BD0000C0
S315080039C0303A000010B50024DFF8DC06007800283D
S315080039D000F06D82DFF8D0060078012836D100F0B5
S315080039E057FD00F0EBFCDFF8CC0600F01DFDDFF814
S315080039F0C80600F019FD00F0DFFC01220100DFF81F
S31508003A00BC06FDF786FE002807D0DFF8B40600F0EE
S31508003A100BFD012000F0FEFC49E2DFF8A80600F0E5
S31508003A2003FDDFF8A40600F0FFFCDFF8A00600F0AF
S31508003A30FBFC0020DFF8981608600020DFF89016D7
S31508003A4048600220DFF86016087030E2DFF8580692
S31508003A500078022840F06681DFF860264FF480710E
S31508003A60DFF87006FEF7B0FADFF8401691F8411253
S31508003A7000290FD0DFF8480600F0D6FC022000F037
S31508003A80C9FCDFF83806FEF723F90020DFF8181618
S31508003A9008700CE200281BD00022DFF83C16DFF87D
S31508003AA0340600F045FA040024B214F1010F0FD1D0
S31508003AB0DFF80C0600F0B8FC032000F0ABFCDFF8DA
S31508003AC0FC05FEF705F90020DFF8DC150870EEE1C5
S31508003AD024B2012CC0F29580DFF8F405406800286E
S31508003AE00BD1DFF8F005D0F88001DFF8E41508609F
S31508003AF024B2DFF8DC05446083E0DFF8D805D0F8A7
S31508003B008001DFF8CC150968DFF8C425526851181A
S31508003B10884208D1DFF8B805406800FA84F0DFF873
S31508003B20B01548606DE0DFF89C0500F07DFCDFF815
S31508003B30AC0500F079FCDFF8A815DFF894054068B5
S31508003B4000F009FBDFF8980500F06EFCDFF8940535
S31508003B5000F06AFCDFF88815DFF874050068000EC7
S31508003B60C0B200F0E6FADFF88015DFF864050068F1
S31508003B70000CC0B200F0DDFADFF87015DFF850056A
S31508003B800068000AC0B200F0D4FADFF86415DFF85E
S31508003B9040050068C0B200F0CCFADFF8440500F032
S31508003BA043FCC3A000F040FCDFF824054168DFF8B9
S31508003BB02005006800F074FC00280FD1DFF8000526
S31508003BC000F032FC052000F025FCDFF8F004FEF7D3
S31508003BD07FF80020DFF8D014087068E1DFF8E40405
S31508003BE000F022FCDFF8E40400F01EFCDFF8E40431
S31508003BF0D0F88001DFF8D814086024B2DFF8D004C2
S31508003C004460DFF8A804D0F84402DFF8A014D1F81D
S31508003C103C12884201D1012000E00020C0B20028F1
S31508003C2000F045810021DFF89404FEF765F80028C6
S31508003C300FD0DFF88C0400F0F7FB042000F0EAFB55
S31508003C40DFF87804FEF744F80020DFF85C14087003
S31508003C502DE1DFF87C04406800285AD0DFF86404B8
S31508003C6000F0E2FBDFF8740400F0DEFBDFF8701406
S31508003C70DFF85C04406800F06EFADFF8640400F0D0
S31508003C80D3FBDFF8600400F0CFFBDFF85414DFF84D
S31508003C9040040068000EC0B200F04BFADFF8481482
S31508003CA0DFF82C040068000CC0B200F042FADFF816
S31508003CB03C14DFF81C040068000AC0B200F039FAA8
S31508003CC0DFF82C14DFF808040068C0B200F031FAF7
S31508003CD0DFF80C0400F0A8FB75A000F0A5FBDFF8E0
S31508003CE0F0034168DFF8E803006800F0D9FB002814
S31508003CF00FD1DFF8CC0300F097FB052000F08AFB14
S31508003D00DFF8B803FDF7E4FF0020DFF89C1308701E
S31508003D10CDE0DFF8B00300F087FB0320DFF8881357
S31508003D200870C4E0DFF880030078032840F0BF80FD
S31508003D30DFF888234FF48071DFF89803FEF744F91B
S31508003D40DFF8681391F8411200290ED0DFF8A403B2
S31508003D5000F06AFB022000F05DFBDFF86003FDF768
S31508003D60B7FF0020D0490870A1E000281AD0DFF874
S31508003D708823DFF86413DFF85C0300F0D9F8040041
S31508003D8024B214F1010F0DD1DFF8700300F04CFBDB
S31508003D90032000F03FFBC948FDF79AFF0020C249FF
S31508003DA0087084E024B2012C4CDBD54800F03CFBBB
S31508003DB0CB4924B2200000F0CEF9C94800F034FB04
S31508003DC0D04800F031FBC649C248D0F88001000E41
S31508003DD0C0B200F0AEF9C449BE48D0F88001000C64
S31508003DE0C0B200F0A6F9C149BA48D0F88001000A65
S31508003DF0C0B200F09EF9BE49B648D0F88001C0B2FC
S31508003E0000F097F9B64800F00FFB29A000F00CFB6C
S31508003E10B94A24B22100AF48D0F8800100F03CFB33
S31508003E2000280CD1A64800F0FFFA062000F0F2FAA6
S31508003E30A248FDF74DFF00209B49087037E0A148CE
S31508003E4000F0F2FA9948D0F844029849D1F83C12A1
S31508003E50884201D1012000E00020C0B2002826D007
S31508003E60A94800F0E1FA00F027FB00280CD1944895
S31508003E7000F0DAFA072000F0CDFA9048FDF728FF9F
S31508003E8000208949087012E08E4800F0CDFA9F4854
S31508003E9000F0CAFA8948FDF71BFF9D4800F0C4FAEE
S31508003EA000208149087000F09AFA00F013FB10BD53
S31508003EB02E2E2E0010B50400207800F03CFB532867
S31508003EC004D1607800F03DFB002801D103200FE003
S31508003ED06078312801D100200AE06078322801D1C3
S31508003EE0012005E06078332801D1022000E0032094
S31508003EF010BD70B504000026A41C200000F044F98B
S31508003F000500AE19A41C200000F03EF986196D1EA6
S31508003F10A41CADB2022DF6DAF6B2F643200000F084
S31508003F2033F9F6B2864201D0002000E0012070BDC8
S31508003F302DE9F04107000C0015005FF00008002C81
S31508003F4001D0002F04D140F26121594800F041F90F
S31508003F503800FFF7AFFF0600F6B2032E01D10020A6
S31508003F60A0E03800FFF7C5FF002802D15FF0FF3058
S31508003F7098E0F6B2002E03D0022E58D027D38FE051
S31508003F80BF1C380000F000F90600BF1C380000F01E
S31508003F90FBF800022060BF1C380000F0F5F8216825
S31508003FA051FA80F02060BF1CB6F10308002D0DD031
S31508003FB0002406E0380000F0E7F8A4B22855BF1C34
S31508003FC0641CA4B20FFA88F84445F3DB68E0BF1C0A
S31508003FD0380000F0D9F80600BF1C380000F0D4F805
S31508003FE000042060BF1C380000F0CEF82168C0B27B
S31508003FF011EB00202060BF1C380000F0C5F82168CE
S3150800400051FA80F02060BF1CB6F10408002D0DD0CF
S31508004010002406E0380000F0B7F8A4B22855BF1C03
S31508004020641CA4B20FFA88F84445F3DB38E0BF1CD9
S31508004030380000F0A9F80600BF1C380000F0A4F804
S3150800404000062060BF1C380000F09EF82168C0B248
S3150800405011EB00402060BF1C380000F095F821687D
S31508004060C0B211EB00202060BF1C380000F08CF8AD
S31508004070216851FA80F02060BF1CB6F10508002DB2
S315080040800DD0002406E0380000F07EF8A4B22855CA
S31508004090BF1C641CA4B20FFA88F84445F3DBFFE79B
S315080040A0404600B2BDE8F081A9200020D40E0020C9
S315080040B0DC7700080C7900089878000804110020BD
S315080040C0647B00086C7B0008307900080C780008CF
S315080040D06C200020601B0020E01C0020447B0008A8
S315080040E03C1F0020007A00083E1F0020401F0020C9
S315080040F0421F002054790008601C002078790008C7
S31508004100E87A00087C7A00081C7A0008947A000885
S315080041106C78000880B5010011F00F003030C9B284
S315080041200A2901DBC01D02E0C0B200F004FAC0B2E1
S3150800413002BD38B504000D002000C0B20009FFF723
S31508004140E9FF287014F00F00FFF7E4FF68700020FD
S31508004150A870280032BD0200491C0A23B2FBF3F2FC
S31508004160002AF9D100220A700200491E0A20B2FB71
S31508004170F0F300FB1320303008700A20B2FBF0F28F
S31508004180002AF2D10800704770B504000025002601
S3150800419009E03038C0B20A2800DBC01FEDB2290199
S315080041A051FA80F5761CF6B2022E0FDAF6B2A05D49
S315080041B000F0C1F9C0B2B0F13001172904D2C0B27B
S315080041C0B0F13A010729E4D2002001E02800C0B284
S315080041D070BD80B500F0BEF9FCE7000080B500F0C0
S315080041E0BDF900F04CFC01203F49087000F084FD41
S315080041F000203D49087000F047FE02203A49087041
S3150800420001BD80B5394800F00BFD012805D1012014
S3150800421035490870354800F0CBF9344800F0B7FD49
S31508004220012805D1002030490870304800F0C0F94F
S315080042302E4800F091FE012805D102202A4908706F
S315080042402A4800F0B5F901BD80B500F04CFE01BD65
S3150800425038B504000D0024480078012804D1290047
S31508004260C9B2200000F08CFC1F480078002804D151
S315080042702900C9B2200000F05DFD1B48007802281D
S3150800428004D12900C9B2200000F036FE00F08AF9F0
S3150800429031BD15480078002805D0022807D004D378
S315080042A0032806D007E0402006E0082004E03F2067
S315080042B002E0002000E0402080B270470A480078FB
S315080042C0002805D0022807D004D3032806D007E023
S315080042D0402006E0082004E03F2002E0002000E03D
S315080042E0402080B270470000DC000020FC1E002041
S315080042F080B500F04EF902BD80B501215D48FEF794
S3150800430027FC012801D1002002E001F014F8012061
S3150800431002BD80B5642000F0E7FF01BD80B500F05E
S31508004320E6FF01BD1CB5040053480078002819D1E2
S3150800433001210420FEF7FAFC4FF4006000900120EA
S315080043408DF8040001208DF8060000208DF807007E
S3150800435002208DF8050069464848FEF7A7FB0120AC
S3150800436045490870E4B2012C05D14FF40061434871
S31508004370FEF7FBFB04E04FF400614048FEF7F3FB51
S3150800438013BD7047704700B5C7B068464FF48C71C7
S3150800439000F0E0FF69463A48FDF778FD002808D1A5
S315080043A00098002805D09DF80800C00601D4012011
S315080043B000E0002047B000BD3148704780B50020B6
S315080043C0304981F828020A222F492E48FDF7A1F91B
S315080043D0002803D101202B4981F8280201BD10B518
S315080043E0284890F82802012802D12648FDF770FCD3
S315080043F0FEF71EFD10F164044021244801F026F85A
S31508004400002803D1FEF714FD8442F5D21C48FDF7B7
S315080044106BFD10BD80B51B4890F82802012802D113
S315080044201848FDF755FC01BD10B50400154890F86D
S315080044302802012819D113492000FDF713FE002888
S3150800444013D500200F4981F828020E48FDF740FCD5
S315080044500BE0217889B20D4800F0F0FF80210B4867
S3150800446000F0F4FF0028F9D0641C20780028F0D169
S3150800447010BD000000000240AA20002000080240EB
S31508004480E07900082C130020F87A00080044004060
S3150800449080B500F0E9FF01BD80B500F0F0FF02BD70
S315080044A080B501F016F802BD80B501F06AF802BDC4
S315080044B080B501F0B0F802BD80B501F024F80028F7
S315080044C001D1002001E001F08BF802BD80B501F0B2
S315080044D0CDF901BD10B5FFF7E7FF002814D0FFF7A7
S315080044E00BFF002810D0FFF7AFFEFEF793FCFFF78F
S315080044F0DFFF0649084006490860FFF7D9FF001D97
S31508004500046801F0B5F9A04710BD000080FFFF1F41
S3150800451008ED00E070B504000D00160005E02878E7
S3150800452020706D1C641C00F015F83000461E80B221
S315080045300028F4D170BDA0F161011A2938BF2038CE
S31508004540704730380A288041C00F704780B5FFF79A
S31508004550E0FE01BD80B5FFF7E1FE01BD0020DFF8F2
S31508004560701408700020DFF8681488640020DFF8EB
S31508004570601481F843000020DFF85414A1F84400C1
S315080045800020DFF84C1488700020DFF844144870C7
S315080045907047DFF83C040078002801D1002000E0CD
S315080045A0012070470020DFF8281481F8430070477F
S315080045B080B50178FF291ED100F091F8DFF81004C4
S315080045C090F84300012802D1102000F07EF8DFF8A9
S315080045D00004B0F9440001280CDB0120DFF8F013D1
S315080045E081F84300DFF8E803B0F94410DFF8E40384
S315080045F000F053F801BDDFF8D813097801294BD12B
S315080046000178C92932D0CC293FD0CF293AD0D02930
S315080046102FD0D12933D0D2292ED0F32917D0F42977
S315080046200FD0F5290AD0F6290ED0FA2912D0FC297E
S3150800463013D0FD2914D0FE2915D029E000F0D9F8A9
S31508004640BCE700F0F9F8B9E700F0C8F8B6E700F0FB
S3150800465019F9B3E700F0AAF8B0E700F0A2F8ADE759
S3150800466000F087F8AAE700F076F8A7E700F03DF92A
S31508004670A4E700F05CF9A1E700F01BF99EE700F05B
S3150800468088F99BE700F099F998E700F0ABF995E708
S31508004690202000F01AF891E7ACE780B589B2FFF759
S315080046A0D7FD01BD10B4002302E00478E318401CCE
S315080046B00C00611E002CF8D1DBB21360012010BC7F
S315080046C070470020C24948707047FE21C04AD17021
S315080046D0BF4908710220BE49A1F84400704780B559
S315080046E0FFF74AF9002803D11020FFF7EEFF31E063
S315080046F0FFF7E7FF0120B6490870FF20B449C870E4
S315080047000020B3490871B248007950F01000B0494A
S3150800471008710020AE494871AD484079AC494871E6
S31508004720FFF7B7FDAA498871FFF7C8FDA849C87100
S31508004730FFF7C4FD80B2000AA54908720120A44902
S3150800474048720120A24988720820A149A1F84400AC
S31508004750FFF79EFE01BD80B500209D490870FFF752
S31508004760B0FFFF209A49C87001209949A1F8440072
S3150800477001BDFF209649C8700020954908719448E4
S3150800478040789349487100209149887100209049E2
S31508004790C87100208E49087206208D49A1F8440088
S315080047A0704780B50020FFF790FF01BDFF208849BC
S315080047B0C8708948864988640020854908710020A0
S315080047C08349487100208249887107208049C1F8C9
S315080047D0070008207E49A1F844007047FF217C4A5B
S315080047E0D17040687A49886401207949A1F8440063
S315080047F0704710B50400FFF74CFD80B2401E617883
S31508004800884203DA2220FFF760FF14E0627892B24A
S315080048106F48816C7148FFF77DFEFF206C49C870B0
S315080048206B48806C61784018694988646078401CD8
S315080048306749A1F8440010BD10B50400FFF729FD2B
S3150800484080B2401E6178884203DA2220FFF73DFFD6
S3150800485017E060685E498864627892B25C48816C49
S315080048605E48FFF757FEFF205949C8705848806CC4
S3150800487061784018564988646078401C5449A1F804
S31508004880440010BD80B5FF21514AD170544A416891
S315080048904F48806CFFF706FF4D49087100204C49C8
S315080048A0487100204A49887108204949A1F84400FE
S315080048B001BD80B5FF204649C870002044490871EB
S315080048C0002043494871FFF7E4FC414988710020FC
S315080048D03F49C87100203E49087200203C49487289
S315080048E007203B49A1F8440001BD10B50400FFF7B5
S315080048F0D0FC621C80B2411E3548806CFFF7CCFDA7
S31508004900002803D13120FFF7E0FE0FE0FF203049F1
S31508004910C870FFF7BEFC2E49896C80B2401E40184D
S315080049202B49886401202A49A1F8440010BD10B516
S315080049300400FFF7AEFC80B2801E6178884203DA75
S315080049402220FFF7C2FE23E0FF202149C87001207C
S315080049501F49A1F844006078002807D1FFF7ACFD8D
S31508004960002802D13120FFF7B0FE11E0A21C6178C1
S315080049701748806CFFF790FD002803D13120FFF718
S31508004980A4FE05E01248806C6178401810498864D6
S3150800499010BD80B541680E48806CFFF781FD002880
S315080049A003D13120FFF791FE06E0FF200849C870C1
S315080049B001200749A1F8440001BD80B5FFF78AFD2B
S315080049C0FF200349C87001200149A1F8440001BD30
S315080049D0E41D0020E71D00207C7B0008E81D002060
S315080049E0EB1D002080B53120FFF76FFE01BD0000EA
S315080049F0F0B4002400E0641CE4B2122C3CD24AF263
S31508004A00104580B2A64EE4B216F81460A44FE4B27C
S31508004A1007EB44077F78BE19761C06FB00F695FB64
S31508004A20F6F706FB1755002DE5D14AF2104580B278
S31508004A309B4EE4B216F81460994FE4B207EB4407AC
S31508004A407F78BE19761C06FB00F695FBF6F50D80F9
S31508004A500D88002DCFD00D88B5F5806FCBDC90483A
S31508004A60E4B210F8140010708D48E4B200EB44006C
S31508004A7040781870012000E00020F0BC704780B52F
S31508004A806B460DF101020DF102014FF4FA70FFF7C2
S31508004A90AFFFC0B2012803D0EE218248FFF799FB89
S31508004AA00020814908608148006850F400407F4929
S31508004AB0086001E0FFF74EFD7C4800680004F9D461
S31508004AC07A48006830F0020078490860774800683C
S31508004AD050F001007549086001E0FFF73BFD744896
S31508004AE00068C007F9D59DF80100401E9DF8001022
S31508004AF0491E090551EA0040BDF80210491E08433F
S31508004B006C490860694800684008400067490860C1
S31508004B1001E0FFF71FFD66480068C007F9D466483C
S31508004B20006850F00100644908606448006840085D
S31508004B304000624908606248006850F00100604918
S31508004B40086000205F49086000205F4908605F48E8
S31508004B500068400840005D4908605D4800684008F4
S31508004B6040005B4908605548006850F00100534909
S31508004B70086051480068400840004F49086001BD78
S31508004B8070B504000D0040F2E17652480068400115
S31508004B9004D44FF4A2714348FFF71BFB4E48006844
S31508004BA010F001004C490860002E06D44A480068F7
S31508004BB050EA46504849086009E026F0004646484B
S31508004BC00068F10051F00401084343490860EDB25A
S31508004BD042480560E078A178090451EA00606178E6
S31508004BE050EA0120217808433D490860E079A17917
S31508004BF0090451EA0060617950EA012021790843E5
S31508004C00384908603448006850F0010032490860A5
S31508004C1001E0FFF79FFC2F4800684001F9D570BDF9
S31508004C200021314A126812F0030F35D02F4A126854
S31508004C30520703D42D4A1268520D04E02B4A126813
S31508004C40D20852F0004240F267639A421ED101210F
S31508004C50274A12680270264A1268120A4270244AC3
S31508004C601268120C8270224A1268120EC270214A09
S31508004C70126802711F4A1268120A42711D4A1268A6
S31508004C80120C82711B4A1268120EC271164800680D
S31508004C9050F02000144A10600800C0B270470000A7
S31508004CA0E87800082877000814640040006400408B
S31508004CB0046400401C640040006600401C66004016
S31508004CC00C660040406600404466004004660040AA
S31508004CD01466004008640040806500408465004012
S31508004CE0886500408C6500400C640040B065004053
S31508004CF0B8650040BC65004000B585B04FF461401A
S31508004D0000900020ADF804000020ADF80600002051
S31508004D10ADF808000020ADF80C000C20ADF80A002C
S31508004D206946524800F01AFB0121504800F078FB0A
S31508004D3005B000BD70B504000D00EDB2412D03DBD2
S31508004D4076214B48FFF745FA2800C0B200F075F8FF
S31508004D50C0B2012803D07A214548FFF73AFA00265F
S31508004D600DE0FFF7F7FBB6B2A05D00F066F8C0B23B
S31508004D70012803D083213E48FFF72BFA761C300022
S31508004D802900C9B280B289B28842EAD370BD10B58B
S31508004D90040038480078002813D1374800F03DF859
S31508004DA0012838D134480078002834D0FEF740F876
S31508004DB03249086000203249087001202D490870E0
S31508004DC029E02D482E4909780844401C00F025F8AA
S31508004DD0012816D12A480078401C29490870284815
S31508004DE0007825490978884215D12548027892B273
S31508004DF024492000FFF78EFB00201E490870012079
S31508004E000AE0FEF715F81D4909686431814202D2A5
S31508004E10002018490870002010BD10B50400202194
S31508004E20124800F013FB012805D1104800F00AFBD0
S31508004E302070012000E0002010BD10B5040080217C
S31508004E400A4800F003FB002801D100200CE0E4B278
S31508004E50210089B2054800F0F1FA8021034800F0E4
S31508004E60F5FA0028F9D0012010BD000000440040E2
S31508004E70A8760008AD200020301E002088200020DB
S31508004E80AC200020311E002080B500F00FF940212B
S31508004E90DFF8100400F01DF9DFF80C140870402143
S31508004EA0DFF8080400F015F9DFF804140870DFF8D5
S31508004EB0F8030078FF2804D0DFF8F4030078FF2809
S31508004EC004D17821DFF8EC03FFF783F9DFF8E8036C
S31508004ED00090DFF8E833DFF8E8230121DFF8E40380
S31508004EE000F0C8FC01BD80B5DFF8D80300F07CFFF0
S31508004EF00020FFF717FA01BD70B504000D00EDB2EA
S31508004F00402D04DB9A21DFF8AC03FFF762F928008D
S31508004F10C0B200F067F8C0B2012804D09E21DFF8BD
S31508004F209403FFF756F900260EE0FFF713FBB6B217
S31508004F30A05D00F057F8C0B2012804D0A721DFF819
S31508004F407403FFF746F9761C30002900C9B280B20F
S31508004F5089B28842E9D370BD10B50400DFF864034E
S31508004F6000F04EFFDFF860030078002812D1DFF862
S31508004F705C0300F02FF801280AD1DFF85003007807
S31508004F80002805D00120D04908700020D0490870B3
S31508004F90002010BDCD48CE4909780844401C00F0D1
S31508004FA019F80128F4D1CA480078401CC849087085
S31508004FB0C7480078C54909788842E9D1C4480278C3
S31508004FC092B2C4492000FFF7A5FA0020BE4908702E
S31508004FD00120DEE780B50100B548007800F0F4F856
S31508004FE0C0B202BD80B50100C9B2AF48007800F072
S31508004FF089F8C0B202BD38B5AB48007800F040F970
S315080050000400E4B2002C25D0E4B2412C00DB402495
S31508005010002512E06946A448007800F0D5F8C0B229
S31508005020012804D04FF49271A248FFF7D2F89DF8F0
S315080050300000A949EDB248556D1C28002100C0B2F0
S31508005040C9B28842E6D3E4B22300A34A81219D4827
S3150800505000F05AFE31BD38B500249A49C0B228225C
S3150800506050430844D0F88C43002510E001F04DFA6F
S31508005070ADB2415D8E48007800F044F8C0B2012810
S3150800508004D040F243118B48FFF7A3F86D1C2800A3
S31508005090210080B289B28842E8D301F036FA0200CC
S315080050A040230121874800F00CFE31BD8B498C4A0C
S315080050B0002004E088744A6118311832401CC0B2D6
S315080050C00028F7D08874002048618448854908601C
S315080050D0704710B4834A1268002A01D1FF200FE0F6
S315080050E0804A126853697F4C236011749060D060BF
S315080050F0002353741060C9B20844401E5060907C67
S3150800510010BC704738B504000D00E4B2022C04DB6D
S315080051104FF4CD716748FFF75CF87048E4B2182180
S3150800512001FB04F10844407C6C49E4B2182202FBF6
S3150800513004F21144097C884201D1002043E0674803
S31508005140E4B2182101FB04F10844C06805706348FD
S31508005150E4B2182101FB04F10844407C401C5F4975
S31508005160E4B2182202FB04F2114448745B48E4B224
S31508005170182101FB04F10844C068401C5749E4B2F1
S31508005180182202FB04F21144C8605448E4B21821FC
S3150800519001FB04F1084440685049E4B2182202FBB6
S315080051A004F21144C96888420CD24C48E4B218216A
S315080051B001FB04F140584949E4B2182202FB04F203
S315080051C01144C860012032BD38B504000D00E4B2B0
S315080051D0022C04DB4FF4DE713648FEF7FAFF3F482F
S315080051E0E4B2182101FB04F10844407C002801D1EF
S315080051F0002044E03948E4B2182101FB04F10844D0
S315080052008068007828703548E4B2182101FB04F15B
S315080052100844407C401E3149E4B2182202FB04F2DD
S31508005220114448742D48E4B2182101FB04F10844DE
S315080052308068401C2949E4B2182202FB04F2114492
S3150800524088602648E4B2182101FB04F10844406846
S315080052502249E4B2182202FB04F211448968884202
S315080052600CD21E48E4B2182101FB04F140581B4930
S31508005270E4B2182202FB04F211448860012032BD10
S3150800528010B50400E4B2022C04DB4FF4EE710948B1
S31508005290FEF79FFF1148E4B2182101FB04F1084408
S315080052A0407C10BD751E0020741E0020B91E00200B
S315080052B0B81E002064770008C000002010000020F7
S315080052C08C000020E0080020AF2000207C1F002072
S315080052D0AE2000207D1F0020BC1F00203C2000209F
S315080052E0542000208C20002016490880704780B57D
S315080052F0FDF79EFD1449096888421BD313480078B8
S31508005300002808D10120114908704FF4805110482F
S31508005310FDF72BFC07E000200C4908704FF480517C
S315080053200B48FDF720FCFDF783FD06490988401860
S315080053300549086001BD80B54FF480510448FDF762
S3150800534012FC01BDA62000207C200020AB200020F6
S3150800535000080240002201F0F1B8000030B585B01F
S3150800536004000D000020002000210021A889002843
S31508005370208A30F44050E98808432082A0892749CA
S315080053800840A9882A8911436A8911430843A081DC
S31508005390A08A30F44070A9890843A0826846FDF7C0
S315080053A059FC1C48844202D01B48844201D1039808
S315080053B000E00298A189090406D5192148432968FD
S315080053C04900B0FBF1F105E0192148432968890035
S315080053D0B0FBF1F16420B1FBF0F00001020964238F
S315080053E003FB1211A289120408D5C90032316422BE
S315080053F0B1FBF2F111F00701084307E00901323168
S315080054006422B1FBF2F111F00F010843208105B0C7
S3150800541030BD00000010014000140140F3E9FFFF11
S31508005420C9B2002904D0818951F40051818104E070
S3150800543081894DF6FF72114081817047C905C90DF2
S31508005440818070478088C005C00D7047002289B2E8
S31508005450B1F5007F0088084201D0012200E0002251
S315080054601000C0B2704700005FF0FF30DFF8EC13A1
S3150800547008605FF0FF30DFF8E8130860704770B522
S3150800548004000D001600200000F0BAF9FF2805D028
S315080054902819401E00F0B4F9FF2801D1002017E0B2
S315080054A0600A4FF400714843DFF8B8130968884268
S315080054B007D12B0032002100DFF8A40300F0E0F842
S315080054C006E02B0032002100DFF8900300F0D8F840
S315080054D070BD70B504000D00200000F091F90600BB
S315080054E02819401E00F08CF9F6B2FF2E02D0C0B281
S315080054F0FF2801D1002005E00100C9B23000C0B282
S3150800550000F03CF970BD80B500200090DFF850032C
S31508005510006810F1010F01D1012031E00098DFF891
S3150800552040134968081800900098CD4989680818FA
S3150800553000900098CA49C968081800900098C84998
S315080055400969081800900098C54949690818009023
S315080055500098C3498969081800900098C049C96924
S31508005560081800900098C04300900098401C0090CE
S315080055706A460421BB48006810F5C470FFF77FFF30
S3150800558002BD0020B749096809680818B5490968BD
S31508005590091D09680818B34909680831096808180F
S315080055A0B04909680C3109680818AE49096810310C
S315080055B009680818AB490968143109680818A9491F
S315080055C00968183109680818A649096811F5C471E7
S315080055D009680818002801D1012000E0002070475A
S315080055E080B59F48006810F1010F06D09C4800F06E
S315080055F08AF8002801D100200CE09848006810F1CC
S31508005600010F06D0954800F07EF8002801D1002049
S3150800561000E0012002BD93480068704780B5CA05BE
S3150800562001D000200BE002688A4201D1012006E081
S3150800563001604FF40072001DFEF76CFF012002BDE9
S3150800564038B504000D008648844208D1834C2900E9
S315080056502000FFF7E3FF002810D100200FE0814863
S315080056600068854203D17E4C7E480568EFE7200036
S3150800567000F049F80028EAD1002000E0200032BDF9
S315080056802DE9F04104000F0015001E00780A4FF4BA
S31508005690007101FB00F8206810F1010F07D141469F
S315080056A02000FFF7BBFF002801D1002029E0206871
S315080056B0404508D041462000FFF7C2FF0400002CF1
S315080056C001D100201DE02068381A2044071DFEF786
S315080056D041FF201D381AB0F5007F0AD318F500716E
S315080056E02000FFF7ADFF0400002C01D1002008E0E0
S315080056F0271D287838707F1C6D1C761E002EE6D173
S315080057000120BDE8F0812DE9F0410400012520685B
S3150800571000F076F8C0B2FF2801D100202CE000F096
S3150800572027FFF32000F0B7FF00F0B8FF012803D1E8
S3150800573000F02EFF00201FE05FF0000801E018F1DE
S315080057400108B8F1800F13D2206810EB880604EB25
S3150800575088004768FEF7FEFE3900300000F075FF46
S31508005760082801D0002503E03068B842E7D00025B4
S3150800577000F00EFF2800C0B2BDE8F08138B504007D
S315080057800D0028002100C0B2C9B2884201D200200B
S3150800579035E020003349097AC0B2884206D3314839
S315080057A090F874002900C9B2884201D2002026E088
S315080057B000F0DEFEF32000F06EFF00F06FFF012818
S315080057C003D100F0E5FE002019E000E0641C280083
S315080057D02100C0B2C9B288420ED3FEF7BBFE022131
S315080057E02148E4B230F8140000F0DBFE0828EDD0BA
S315080057F000F0CEFE002002E000F0CAFE012032BD15
S3150800580038B50400002500E06D1CEDB20A2D21D242
S31508005810FEF7A0FE1348EDB20C2101FB05F1405836
S315080058208442F1D30F48EDB20C2101FB05F1405833
S315080058300C49EDB20C2202FB05F21144496808181E
S315080058408442E1D20748EDB20C2101FB05F1084478
S31508005850007A00E0FF2032BD000000005815002045
S315080058605C170020B87500083C78000872B67047C7
S3150800587062B67047F8B504000D0016001F00200038
S31508005880FDF7FCFF200000F014F8C4F8E47506984C
S31508005890C4F8E805C4F8EC652900C9B2200000F090
S315080058A070F9D4F8E805006880472000FEF73CF850
S315080058B0F1BD002070471CB504006946200001F0C0
S315080058C0EFF99DF8000010F01F00C0B2002803D0C1
S315080058D002280BD005D30EE06946200000F01AFF17
S315080058E010E06946200000F041FF0BE06946200001
S315080058F000F063FF06E09DF8000010F0800120002C
S3150800590000F022FA002016BD10B50400C9B200291D
S3150800591034D14FF45D70204494F8111103293CD119
S315080059208168C269914217D2C1698268891AC161C0
S31508005930E178012903D1C16882681144C160C1694F
S315080059408268914201D2C26900E0826892B2C16857
S31508005950200001F021FA20E0D4F8E40500690028C7
S3150800596008D094F81201032804D12000D4F8E415CD
S3150800597009698847200001F01AFA0EE0D4F8E40510
S315080059808069002809D094F81201032805D1C9B204
S315080059902000D4F8E42592699047002010BD38B558
S315080059A00400C9B2002951D14FF48E7004EB0005EA
S315080059B094F8110102283ED1A868E969884211D2F3
S315080059C0E869A968401AE861E078012803D1E8681F
S315080059D0A9680844E860EA6992B2E968200001F01B
S315080059E0D0F928E0286AA968B0FBF1F201FB120099
S315080059F000280FD1286AA96888420BD3286A696AE1
S31508005A00884207D200220021200001F0BAF90020BE
S31508005A10686210E0D4F8E405C068002808D094F855
S31508005A201201032804D12000D4F8E415C968884770
S31508005A30200001F0CEF994F81601012815D12000AE
S31508005A4000F015F8002084F816010EE0D4F8E405F5
S31508005A504069002809D094F81201032805D1C9B273
S31508005A602000D4F8E42552699047002032BD034946
S31508005A7009680069416000207047000094200020F2
S31508005A8010B50400002340220021200000F0C8F8C9
S31508005A90002340228021200000F0C2F8012084F86B
S31508005AA01201A078D4F8E81549688847002010BD87
S31508005AB010B50400D4F8E8050069804794F8130186
S31508005AC084F81201032084F81201002010BD80B565
S31508005AD090F8121180F81311042180F81211D0F8E9
S31508005AE0E805C0688047002002BD80B5D0F8E415F7
S31508005AF0C969002903D0D0F8E415C9698847002088
S31508005B0002BD10B50400C9B22000D4F8E425126815
S31508005B109047D4F8E80580688047002010BD80B516
S31508005B20C9B2D0F8E42552689047002002BD80B576
S31508005B30D0F8E415096A8847002002BD80B5D0F878
S31508005B40E415496A8847002002BD10B50400D4F858
S31508005B50E80540698047012084F81501002010BD3A
S31508005B6010B50400D4F8E8058069804700212000B4
S31508005B70D4F8E42552689047002084F815010020DF
S31508005B8010BD10B50400C9B22000FDF7D1F90120F7
S31508005B9084F81201002084F81401002013E028215B
S31508005BA001FB00F121444FF48E72114401224A7020
S31508005BB00870C8800022CA7040228A600022CA6023
S31508005BC000224A61401C61788842E8D3002013E02D
S31508005BD0282101FB00F121444FF45D721144002293
S31508005BE04A700870C8800022CA7040228A60002263
S31508005BF0CA6000224A61401C61788842E8D32000C6
S31508005C00FDF767FA2000FDF700FA00212000FDF7EE
S31508005C10B3FA2000FDF7EAFA2000FDF74EFA10BDA8
S31508005C2038B5C9B20C0609D5C9B211F07F042825C2
S31508005C306C4304444FF48E752C4408E0C9B211F045
S31508005C407F0428256C4304444FF45D752C4411F0F9
S31508005C507F052570C9B2C909617092B2A260E37066
S31508005C606178002901D02178E180DBB2022B01D1CD
S31508005C70002121712100FDF7DDFB002032BD80B532
S31508005C80C9B20A0609D5C9B211F07F0228235A43B8
S31508005C9002444FF48E731A4408E0C9B211F07F0229
S31508005CA028235A4302444FF45D731A4411F07F03C4
S31508005CB01370C9B2C90951701100FDF7F4FB002031
S31508005CC002BD38B50C00E4B214F07F0128256943FB
S31508005CD001444FF45D752944CA609BB24B610023A9
S31508005CE08B6100234B7014F07F030B70C378012B74
S31508005CF000D10A610A78002A02D1FDF7B1FC01E059
S31508005D00FDF7FCFB002032BD38B5C9B211F07F049F
S31508005D1028256C4304444FF48E752C440125657080
S31508005D2011F07F012170E26022610021A1616361A7
S31508005D302178002903D12100FDF792FC02E0210019
S31508005D40FDF7DCFB002032BD80B5C9B20A0609D5CD
S31508005D50C9B211F07F0228235A4302444FF48E73C6
S31508005D601A4407E0C9B2282202FB01F202444FF4A2
S31508005D705D731A440123937011F07F031370C9B23F
S31508005D80C90951701100FDF7FEFC002002BD80B55F
S31508005D90C9B20A0609D5C9B211F07F0228235A43A7
S31508005DA002444FF48E731A4407E0C9B2282202FB54
S31508005DB001F202444FF45D731A440023937011F004
S31508005DC07F031370C9B2C90951701100FDF7F9FCB8
S31508005DD0002002BD0022C9B261F30A1201690968EE
S31508005DE0114300690160704780B50169496851F03F
S31508005DF00201006941600320FDF7A3FD01BD000013
S31508005E0070B5040000262000FDF7D6F900286FD0EB
S31508005E102000FDF7DBF90500002D01D1002068E020
S31508005E20C5F3C040002803D0200000F060F90643FF
S31508005E30C5F38040002803D0200000F0E1F80643AF
S31508005E40C5F34000002804D0002050F00200E168A5
S31508005E504861E80F002803D0200000F06CF80643DC
S31508005E60C5F3C020002803D0200000F088F80643B8
S31508005E70C5F3C000002803D0200000F09CF90643B3
S31508005E80C5F30010002803D0200000F0A2F906434D
S31508005E90C5F30030002803D0200000F02EFA064390
S31508005EA0C5F34030002803D0200000F07AFA0643F4
S31508005EB0C5F30050002803D0200000F097FA0643E7
S31508005EC0C5F34050002803D0200000F09DFA064391
S31508005ED0C5F38070002803D0200000F00BF80643B5
S31508005EE0C5F38000002803D0200000F012F806430E
S31508005EF0300070BD10B504002000DFF828150968C9
S31508005F00496A8847002050F08040E16848610120CE
S31508005F1010BD38B50400E0684568C5F38000002860
S31508005F2005D02000DFF8FC140968896A8847E0680C
S31508005F304560012032BD10B50400A07A002808D0BB
S31508005F40D4F80C0130F0020040084000D4F80C11D7
S31508005F500860002050F001002169496831EA000014
S31508005F60216948602000DFF8BC14096889698847F8
S31508005F70002050F00040E1684861012010BD10B5CE
S31508005F8082B0040000208DF8000094F812018DF804
S31508005F9000002000DFF88C140968496988472069E1
S31508005FA08168002050F40060E2685061A07A0028F9
S31508005FB024D0C80722D594F8150101281ED19DF8CA
S31508005FC0000003281AD1002050F00100D4F80C1163
S31508005FD009680143D4F80C21116050F00200D4F886
S31508005FE00C1109680843D4F80C110860DFF8380466
S31508005FF0006850F00600DFF830140860012016BD6E
S31508006000F8B50400002500272000FDF70AFC060065
S3150800601069E0F00765D52900C9B2200000F006FA44
S315080060200700F80722D50120A8402169496B31EA03
S31508006030000021694863002757F0010704EB850033
S31508006040806987602900C9B22000DFF8D823126862
S3150800605052689047E078012808D1002D06D194F8B7
S315080060601101042802D12000FDF7E2FBC7F3C000A6
S31508006070002806D0002757F0080704EB850080693A
S315080060808760C7F30010002806D0002757F01007CE
S3150800609004EB850080698760C7F38010002806D066
S315080060A0002757F0400704EB850080698760C7F32F
S315080060B04000002806D0002757F0020704EB8500A9
S315080060C080698760C7F3C01000280AD0290020001D
S315080060D000F0CDF8002757F0800704EB85008069AB
S315080060E087606D1C7608002E93D10120F2BDF8B5A5
S315080060F00400002500272000FDF782FB060056E075
S31508006100F00752D52900C9B22000FDF780FB070029
S31508006110F8072FD5002757F0010704EB8500406DD7
S315080061208760E078012812D104EB8500406D00698C
S31508006130282101FB05F12144D1F87C134003400BCB
S31508006140081A282101FB05F12144C1F88C0329000E
S31508006150C9B22000B34A126812689047E07801284D
S3150800616008D1002D06D194F81101052802D1200086
S31508006170FDF75EFBC7F34000002806D0002757F05E
S31508006180020704EB8500406D8760C7F3C00000284E
S315080061900BD02000A349096889688847002757F06B
S315080061A0080704EB8500406D87606D1C7608002E95
S315080061B0A6D10120F2BD10B504002000994909684E
S315080061C0C9688847002050F00800E1684861012046
S315080061D010BDF8B50400002555F01005E068806983
S315080061E0A843E1688861E068066A16F00F0028216E
S315080061F0484320444FF45D7100EB0107700C10F022
S315080062000F00012808D0022807D003281AD004282E
S3150800621019D0062818D023E022E03009400510D00E
S31508006220C6F30A1292B2F9682000FCF76DFEF86808
S31508006230C6F30A110844F860B869C6F30A110818C3
S31508006240B8610DE00CE00BE0082204F2CC51200006
S31508006250FCF75AFEB869C6F30A110818B861FFE7D1
S31508006260E06880692843E16888610120F2BD2DE96C
S31508006270F04104000D0000270020282000FB05F04F
S3150800628020444FF48E7100EB01067069B169471A14
S31508006290B068B84200D2B768F81C5FEA900804EB09
S315080062A08500806980691BE07069B169471AB06822
S315080062B0B84200D2B768F81C5FEA90083B009BB268
S315080062C02A00D2B2F1682000FCF701FEF0683844D3
S315080062D0F060B0693818B06104EB850080698069A0
S315080062E080B2804506D2B0697169884202D2706967
S315080062F00028D9D10120BDE8F081F8B504000021B5
S315080063000025002600270020002051F00101206901
S31508006310406888432169486000212000FCF7E6FEB2
S3150800632000200AE004EB80018969FF228A6004EBF9
S315080063308001496DFF228A60401C61788842F1D34A
S315080063405FF0FF3021698861012060F30F050120A5
S3150800635060F31F452069C56156F0080656F0010628
S3150800636056F002062069466157F0010757F00807FC
S3150800637057F00207206907612069006830F4FE605B
S31508006380216908602000FDF753FA002050F4805078
S31508006390E16848612000234909680969884701209E
S315080063A0F2BD38B504002000FDF71FF8E068C5689F
S315080063B02000FDF704F8032808D10020A0704FF448
S315080063C00070A080092060F38D2506E00120A070EA
S315080063D04020A080052060F38D25E068C560002078
S315080063E050F40050E1684861012032BD38B5040018
S315080063F0002520000B490968C969884755F48015A6
S31508006400E0684561012032BD38B50400002520004A
S3150800641004490968096A884755F40015E068456122
S31508006420012032BD8800002010ED00E002691269E3
S3150800643003695B6BCB40DB0113F080031A43C9B2D7
S3150800644000EB8100806980681040704710B5040031
S315080064500223402281212000FFF7E2FB022340228B
S3150800646001212000FFF7DCFB40232F4A01212000F1
S31508006470FFF727FC002010BD10B50400812120007D
S31508006480FFF7FDFB01212000FFF7F9FB002010BDF7
S3150800649010B51722254B0C7814F0600F27D14C78CD
S315080064A0062C04D00A2C14D00B2C17D01FE04C88CD
S315080064B0A4B2240AA4B2212C06D11D4BCA88182AD4
S315080064C001DB172200E0CA8892B2190000F045FCE9
S315080064D00DE00122174900F040FC08E08A78002AFE
S315080064E003D188781349086001E000F0FBFB00201F
S315080064F010BD80B5FEF77FFD002002BD80B50800FF
S31508006500C0B2FEF7A8FD002002BD0748704780B557
S3150800651090F81201032801D1FEF76DFD002002BD97
S315080065202020088004487047FC1F002045000020F2
S315080065304E000020902000203C00002000B500BF3F
S31508006540130096469446103928BFA0E80C50FAD88E
S315080065505FEA417C28BF0CC048BF40F8042BC90736
S3150800656028BF20F8022B48BF00F8012B00BD000009
S31508006570DFF864010068002809D5DFF86001DFF854
S3150800658060110860DFF85C01DFF854110860704795
S31508006590DFF84401006850F00040DFF83C1108605D
S315080065A0704738B5040000250820C9B2002901D172
S315080065B000250DE0C9B2012902D14FF4807507E024
S315080065C0C9B2022902D14FF4007501E04FF44075B3
S315080065D000F08CF8C0B2082835D1DFF8FC00006856
S315080065E030F44070DFF8F0100860DFF8EC0000685F
S315080065F02843DFF8E4100860DFF8DC00006830F0B4
S31508006600F800DFF8D4100860DFF8CC00006854F012
S3150800661002010843DFF8C0100860DFF8BC00006814
S3150800662050F48030DFF8B010086000F05FF82A49AF
S31508006630096831F00201284A11602749096831F0D2
S31508006640F801254A1160C0B232BD38B504000D0004
S31508006650082000F04BF8C0B208281AD11E48006876
S3150800666030F440701C4908601B48006850F40070FC
S31508006670194908601848006850F001001649086072
S31508006680256000F033F81449096849084900124A98
S315080066901160C0B232BD144908607047082012481C
S315080066A00068C00301D5012013E00F480068C00642
S315080066B001D505200DE00C48006810F0EF0F01D059
S315080066C0062006E008480068800701D5072000E094
S315080066D00820C0B270470000103C024023016745FD
S315080066E0043C0240AB89EFCD0C3C024080B5082043
S315080066F08DF80000FFF7D2FF8DF8000003E0FFF7E2
S31508006700CDFF8DF800009DF800000128F7D09DF810
S31508006710000002BD10B500244A78002A18D0012AC4
S315080067201CD0032A17D0052A09D0062A04D0082A1D
S315080067300BD0092A06D014E000F0F4F813E000F0B4
S3150800674083F910E000F0ACF90DE000F009FA0AE070
S3150800675000F023FA07E000F03BFA04E000F086FABE
S3150800676001E000F0BFFA2000C0B210BD70B5040009
S315080067700D00002694F81201032817D1287902285B
S315080067800FDA29002000D4F8E42592689047E888B3
S3150800679000280AD1F6B2002E07D1200000F007FB28
S315080067A003E02900200000F09DFA03E029002000FC
S315080067B000F098FA3000C0B270BD70B505000E0042
S315080067C00024B1887078002860D0012830D00328CA
S315080067D040F0A58095F81201022802D003280BD0B4
S315080067E021E0C9B2002906D0C9B2802903D0C9B2AE
S315080067F02800FFF7A9FA1AE07088002809D1C9B25B
S31508006800002906D0C9B2802903D0C9B22800FFF7EB
S315080068109BFA31002800D5F8E425926890472800AD
S3150800682000F0C5FA03E03100280000F05BFA76E0D4
S3150800683095F81201022802D003280BD021E0C9B22C
S31508006840002906D0C9B2802903D0C9B22800FFF7AB
S315080068507BFA1AE07088002812D1C9B200290CD038
S31508006860C9B2802909D0C9B22800FFF790FA3100C9
S315080068702800D5F8E42592689047280000F097FA92
S3150800688003E03100280000F02DFA48E095F81201DF
S31508006890022802D003280BD03CE0C9B2002906D052
S315080068A0C9B2802903D0C9B22800FFF74DFA35E0EE
S315080068B0C9B2080613D5C9B211F07F00282148438A
S315080068C0284490F81E01002804D00120DFF8881318
S315080068D0086018E00020DFF88013086013E0080657
S315080068E011D4C9B2282000FB01F0284490F8760399
S315080068F0002804D00120DFF86013086003E00020B8
S31508006900DFF8541308600222DFF84C13280000F061
S3150800691024FA03E03100280000F0E4F9FFE720003C
S31508006920C0B270BD38B504000D00688880B2000A90
S31508006930C0B2012808D0022827D0032830D006285C
S3150800694069D007286CD070E06946A078D4F8EC25A1
S3150800695012689047E988402903D094F81211012952
S3150800696002D10821ADF80010BDF8001000296AD040
S31508006970E988002967D0BDF80010EA88914259D203
S31508006980BDF80010ADF8001057E06946A078D4F8B5
S31508006990E425926A904702214170C4F8F005E3E7BE
S315080069A0A878002808D0022814D00CD304281FD0B1
S315080069B017D3052823D029E06946A078D4F8EC2512
S315080069C052689047D0E76946A078D4F8EC259268D3
S315080069D09047F7E76946A078D4F8EC25D26890473F
S315080069E0F0E76946A078D4F8EC2512699047E9E7FC
S315080069F06946A078D4F8EC2552699047E2E76946DB
S31508006A00A078D4F8EC2592699047DBE729002000A6
S31508006A1000F068F917E02900200000F063F912E099
S31508006A202900200000F05EF90DE02900200000F0A2
S31508006A3059F908E0E988ADF80010BDF80020010012
S31508006A40200000F08AF931BD38B50400888800288E
S31508006A5022D1C88800281FD1887810F07F0594F8BD
S31508006A601201032803D1200000F03CF917E084F84E
S31508006A7014512900C9B22000FFF7ACF9200000F034
S31508006A8096F9EDB2002D03D0022084F8120106E033
S31508006A90012084F8120102E0200000F023F931BD3C
S31508006AA010B5040048886D4A10706C4800780228B2
S31508006AB003DB200000F016F951E094F812010228D1
S31508006AC002D0032818D047E06448007800280FD081
S31508006AD06248007884F81001032084F812015F48A0
S31508006AE001782000FFF70DF8200000F060F902E0B9
S31508006AF0200000F05CF932E05848007800280FD1F1
S31508006B00022084F812015548007884F81001534889
S31508006B1001782000FFF703F8200000F048F91AE092
S31508006B204E48007894F81011884211D094F8101144
S31508006B302000FEF7F4FF4948007884F8100147481A
S31508006B4001782000FEF7DDFF200000F030F902E0B2
S31508006B50200000F02CF902E0200000F0C3F810BD78
S31508006B6080B5CA88012A02D000F0BCF814E090F873
S31508006B701221022A02D0032A05D00BE00122384945
S31508006B8000F0EBF808E001224FF48871014400F0A8
S31508006B90E4F801E000F0A6F801BD80B590F81221EE
S31508006BA0921E012A11D801212E4A1160D0F8181117
S31508006BB0002905D02B49096851F00201294A1160BC
S31508006BC00222284900F0C9F801E000F08BF801BD5F
S31508006BD010B504000022488801280BD10120C4F80A
S31508006BE018012000D4F8E42592689047200000F0A8
S31508006BF0DEF830E0488802282DD1087900062AD127
S31508006C0020694068898889B20A0AD2B2012A07D05F
S31508006C1019D3032A0CD007D3052A11D00CD312E0B6
S31508006C20012161F306100EE0022161F306100AE065
S31508006C30032161F3061006E0042161F3061002E061
S31508006C40052161F3061008490860012084F8160139
S31508006C50200000F0ACF810BD98200020B0200020DD
S31508006C609C200020A02000209420002010B50400BD
S31508006C7094F81201801E01280ED8488801280AD1E6
S31508006C800020C4F818012000D4F8E425926890473B
S31508006C90200000F08CF802E0200000F023F810BD78
S31508006CA090F8CC250A7090F8CD254A7090F8CE2534
S31508006CB090F8CF351B029A184A8090F8D02590F89C
S31508006CC0D1351B029A188A8090F8D22590F8D335C8
S31508006CD01B029A18CA80C988C0F84011012180F899
S31508006CE01111704710B5040080212000FFF72CF819
S31508006CF000212000FFF728F82000FCF799FD10BDB9
S31508006D00F8B504000D0017000026002C1AD0200044
S31508006D1000F019F84000801C38803888F6B2A8556B
S31508006D20761C0320F6B2A855761C08E02078F6B241
S31508006D30A855641C761C0020F6B2A855761C207847
S31508006D400028F3D1F1BD002101E0491C401C02785E
S31508006D50002AFAD10800C0B2704710B5002492B2D2
S31508006D60C0F83C2192B2C0F83821022380F81131CC
S31508006D7092B213000A000021FEF7C6FF2000C0B237
S31508006D8010BD10B5002492B213000A000021FEF7C8
S31508006D90BBFF2000C0B210BD10B5002413009BB283
S31508006DA00A000021FEF78DFF2000C0B210BD38B5DD
S31508006DB004000025042084F8110100230022002184
S31508006DC02000FEF7A1FF2000FCF732FD2800C0B224
S31508006DD032BD38B504000025052084F811010023CA
S31508006DE0002200212000FEF76CFF2000FCF720FDA2
S31508006DF02800C0B232BD000061001A03E000170384
S31508006E00F8000703FF000100780100013001320194
S31508006E100601390110014A012E0179010601800196
S31508006E204D004302810182018201840184018601A9
S31508006E308701870189018A018B018B018D018E01EA
S31508006E408F0190019101910193019401F601960138
S31508006E509701980198013D029B019C019D01200222
S31508006E609F01A001A001A201A201A401A401A601FB
S31508006E70A701A701A901AA01AB01AC01AC01AE01AA
S31508006E80AF01AF01B101B201B301B301B501B5015B
S31508006E90B701B801B801BA01BB01BC01BC01BE010A
S31508006EA0F701C001C101C201C301C401C501C40182
S31508006EB0C701C801C701CA01CB01CA01CD0110012A
S31508006EC0DD0101008E01DE011201F3010300F1016B
S31508006ED0F401F401F8012801220212013A0209001C
S31508006EE0652C3B023B023D02662C3F0240024102F2
S31508006EF0410246020A0153024000810186015502F9
S31508006F0089018A0158028F015A0290015C025D02CA
S31508006F105E025F02930161026202940164026502E5
S31508006F2066026702970196016A02622C6C026D027C
S31508006F306E029C01700271029D01730274029F0128
S31508006F4076027702780279027A027B027C02642C46
S31508006F507E027F02A60181028202A90184028502BD
S31508006F6086028702AE014402B101B20145028D02D2
S31508006F708E028F0290029102B7017B030300FD0384
S31508006F80FE03FF03AC0304008603880389038A0310
S31508006F90B1031103C2030200A303A303C403080336
S31508006FA0CC0303008C038E038F03D8031801F20366
S31508006FB00A00F903F303F403F503F603F703F703EB
S31508006FC0F903FA03FA033004200350041007600497
S31508006FD022018A043601C1040E01CF040100C0044F
S31508006FE0D0044401610526040000000080B5484825
S31508006FF0006850F47000464908604648006850F03A
S315080070000100444908600020434908604148006877
S31508007010424908403F4908604148424908603D489E
S31508007020006830F480203B49086000203E4908602B
S3150800703000F005F85FF000603C49086001BD82B0C9
S3150800704000200190002000903248006850F48030FB
S31508007050304908602F48006810F400300090019805
S31508007060401C01900098002803D10198B0F5A06F44
S31508007070F0D128480068800302D50120009001E07D
S3150800708000200090009801283ED12948006850F059
S315080070908050274908602748006850F44040254931
S315080070A008601D4800681C4908601B48006850F4C1
S315080070B00040194908601848006850F4A05016495D
S315080070C008601D48174908601248006850F080702B
S315080070D0104908600F4800688001FBD540F205603A
S315080070E0164908600C480068800880000A4908604C
S315080070F00948006850F00200074908600648006819
S3150800710010F00C000828F9D102B070470000000002
S3150800711088ED00E00038024008380240FFFFF6FE1E
S3150800712010300024043802400C38024008ED00E014
S31508007130403802400070004008544007003C0240B6
S3150800714080B500F005F800F08FF800F09DF8FCE730
S3150800715000B583B001210120FBF7E8FD012000906E
S3150800716000208DF8040000208DF8070002208DF815
S31508007170050069463948FBF799FC01215FF40030A0
S31508007180FBF7F4FD01210120FBF7D0FD07220221C0
S315080071903248FBF7ECFC072203213048FBF7E7FCF3
S315080071A000208DF8060001208DF8070002208DF8D2
S315080071B004000420009002208DF80500694627483F
S315080071C0FBF774FC02208DF804000820009069463D
S315080071D02248FBF76BFC01210220FBF7A7FD0922D9
S315080071E008211F48FBF7C3FC092209211C48FBF7A5
S315080071F0BEFC4FF44070009002208DF80400022077
S315080072008DF8050000208DF8060001208DF807008E
S3150800721069461348FBF74AFC01215FF00070FBF74B
S31508007220A5FD01210420FBF781FD4FF48050009055
S3150800723001208DF8040000208DF8060001208DF845
S31508007240070002208DF8050069460648FBF72EFC64
S315080072504FF480510348FBF786FC07BD0000024047
S31508007260000402400008024080B5FDF72FF9FDF73B
S315080072706DF9FBF7BFFDFDF70BF9FCF769FBFCF7AA
S31508007280ADFF00F00DF801BD80B5FDF763F9FBF71A
S31508007290C5FDFCF797FBFCF7B4FF00F00CF801BD41
S315080072A080B5012013490870FBF7C2FD1249086032
S315080072B000F001F801BD80B5FDF71AF8012818D0CD
S315080072C0FCF75AFB002814D00A480078012810D188
S315080072D0FBF7AEFD0849096811F5FA61884208D33B
S315080072E0002004490870FCF750FB002801D1FDF77F
S315080072F0F1F801BDA820002074200020C700FC007A
S31508007300E900E200E400E000E500E700EA00EB003F
S31508007310E800EF00EE00EC00C400C500C900E60076
S31508007320C600F400F600F200FB00F900FF00D600E4
S31508007330DC00A200A300A500A7209201E100ED0051
S31508007340F300FA00F100D100AA00BA00BF0010232A
S31508007350AC00BD00BC00A100AB00BB009125922586
S31508007360932502252425612562255625552563255D
S31508007370512557255D255C255B25102514253425C3
S315080073802C251C2500253C255E255F255A255425D8
S3150800739069256625602550256C2567256825642599
S315080073A0652559255825522553256B256A251825FF
S315080073B00C25882584258C2590258025B103DF009A
S315080073C09303C003A303C303B500C403A60398032A
S315080073D0A903B4031E22C603B50329226122B100FC
S315080073E06522642220232123F7004822B0001922AF
S315080073F0B7001A227F20B200A025A0007D1D01003B
S31508007400632C001E9601A01E5A01001F0806101FB5
S315080074100606201F0806301F0806401F0606511FCD
S315080074200700591F521F5B1F541F5D1F561F5F1F02
S31508007430601F0806701F0E00BA1FBB1FC81FC91F92
S31508007440CA1FCB1FDA1FDB1FF81FF91FEA1FEB1F26
S31508007450FA1FFB1F801F0806901F0806A01F0806B4
S31508007460B01F0400B81FB91FB21FBC1FCC1F0100F4
S31508007470C31FD01F0206E01F0206E51F0100EC1F0E
S31508007480F21F0100FC1F4E2101003221702110025B
S31508007490842101008321D0241A05302C2F04602C66
S315080074A00201672C0601752C0201802C6401002D4F
S315080074B0260841FF1A030000809A45418E418F80B5
S315080074C04545454949498E8F9092924F994F555552
S315080074D059999A9B9C9D9E9F41494F55A5A5A6A73C
S315080074E0A8A9AAABACADAEAFB0B1B2B3B4B5B6B796
S315080074F0B8B9BABBBCBDBEBFC0C1C2C3C4C5C6C786
S31508007500C8C9CACBCCCDCECFD0D1D2D3D4D5D6D775
S31508007510D8D9DADBDCDDDEDFE0E1E2E3E4E5E6E765
S31508007520E8E9EAEBECEDEEEFF0F1F2F3F4F5F6F755
S31508007530F8F9FAFBFCFDFEFF122008801648704792
S31508007540042008801548704780B50A001449154874
S31508007550FFF7D6FB124802BD80B50A00104912484B
S31508007560FFF7CEFB0E4802BD80B50A000C490F484E
S31508007570FFF7C6FB0A4802BD80B50A0008490C4851
S31508007580FFF7BEFB064802BD80B50A000449094854
S31508007590FFF7B6FB024802BDA8000020BC00002089
S315080075A0E41C0020C47A0008087B0008187B000841
S315080075B0747B0008AC7A00080080000800400000D0
S315080075C00200000000C000080040000003000000A0
S315080075D00000010800000100040000000000020885
S315080075E00000020005000000000004080000020078
S315080075F00600000000000608000002000700000060
S3150800760000000808000002000800000000000A0840
S31508007610000002000900000000000C08000002003B
S315080076200A00000000000E08000002000B0000001F
S31508007630F0B4016844688368014401EB5402E40726
S3150800764048BF4B44914202D1F0BC0C30704711F848
S31508007650015B15F0030604BF11F8014BE61C2C0963
S315080076600F2C07D111F8014B0F3403E011F8017BF9
S3150800767003F8017B761EF9D1002CE3D0AD0811F88A
S31508007680016B05F00305032D08BF11F8015B06EB36
S3150800769005256D42A41C1D44D4D015F8016B03F8CA
S315080076A0016B641EF9D1CDE7433A5C576F726B5C88
S315080076B0736F6674776172655C4F70656E424C5481
S315080076C05C5461726765745C536F757263655C417F
S315080076D0524D434D345F53544D333246345C7561D5
S315080076E072742E630000000019E050F8041BCB07E3
S315080076F044BFA9F101035918121F0023042A41F8AF
S31508007700043BF9D25FEA827C0B4604D54FF0000CA5
S31508007710A1F800C09B1CD10744BF0021197050F87E
S31508007720042B002AE1D17047433A5C576F726B5CB1
S31508007730736F6674776172655C4F70656E424C5400
S315080077405C5461726765745C536F757263655C41FE
S31508007750524D434D345F53544D333246345C636166
S315080077606E2E6300433A5C576F726B5C736F667478
S31508007770776172655C4F70656E424C545C546172F9
S315080077806765745C536F757263655C41524D434D12
S31508007790345F53544D333246345C7573622E63003E
S315080077A07047C0B2002802D0012801D001E000E0ED
S315080077B0FFE77047704780B5FCF7E3FD01BD80B56C
S315080077C0FCF7E0FD01BD80B50120FCF7ABFD01BD6E
S315080077D080B50020FCF7A6FD01BD0000433A5C57C2
S315080077E06F726B5C736F6674776172655C4F7065F8
S315080077F06E424C545C5461726765745C536F757263
S3150800780063655C66696C652E63000000506172737F
S31508007810696E67206669726D776172652066696C44
S315080078206520746F2064657465637420657261737E
S315080078306520626C6F636B732E2E2E0000000800A5
S3150800784010001800200028003000380040004800CA
S31508007850500058008000880090009800A000A800FA
S31508007860B000B800C000C800D000D8004669726DE4
S3150800787077617265207570646174652073756363DA
S3150800788065737366756C6C7920636F6D706C65745F
S3150800789065640A0D000000004F70656E696E67200A
S315080078A06669726D776172652066696C6520666FB8
S315080078B0722072656164696E672E2E2E00000000C4
S315080078C010B5074979441831064C7C44163404E04F
S315080078D00A68081D114488470146A142F8D110BD1F
S315080078E0E0000000FC00000005020602060307038C
S315080078F00803090309040A040B040C040C050D0506
S315080079000E050F050F061006100710084669726D5A
S31508007910776172652075706461746520726571752A
S315080079206573742064657465637465640A0D000084
S315080079305374617274696E67207468652070726F1B
S315080079406772616D6D696E672073657175656E63C3
S31508007950650A0D0052656164696E67206C696E651B
S315080079602066726F6D2066696C652E2E2E45525202
S315080079704F520A0D00000000496E76616C6964205A
S31508007980636865636B73756D20666F756E642E2EFE
S315080079902E4552524F520A0D000000004EF68851ED
S315080079A0CEF20001086840F470000860BFF34F8FFC
S315080079B0BFF36F8F4FF00070E1EE100A70470000BA
S315080079C029FDFFFFD4170000E00800200000000092
S315080079D061FCFFFF1C030000780100000000002086
S315080079E02F64656D6F70726F675F6F6C696D657810
S315080079F05F73746D3332703430352E73726563007D
S31508007A002062797465732066726F6D206D656D6F7F
S31508007A10727920617420307800000000577269740A
S31508007A20696E672070726F6772616D20636865633F
S31508007A306B73756D2E2E2E0000F00BF8002801D002
S31508007A40FFF73EFF0020AFF30080FFF779FB00F059
S31508007A5002F80120704700F001B8000007463846D2
S31508007A6000F002F8FBE7000080B5AFF30080024A99
S31508007A7011001820ABBEFBE72600020020627974CD
S31508007A80657320746F206D656D6F7279206174203F
S31508007A9030780000436C6F73696E67206669726D93
S31508007AA0776172652066696C650A0D0057696E55BF
S31508007AB053422042756C6B20496E74657266616329
S31508007AC06500000057696E5553422042756C6B205D
S31508007AD0446576696365000001030507090E1012FF
S31508007AE01416181C1E00000050726F6772616D6DC7
S31508007AF0696E6720000000002F626F6F746C6F67F5
S31508007B002E747874000000004F70656E424C542045
S31508007B105573657200000000303030303030303038
S31508007B2030353043000000000148804701480047CF
S31508007B30ED6F0008517B0008222A3A3C3E3F7C7FC5
S31508007B400000000045726173696E6720000000003E
S31508007B50AFF30080FFF722FFFFF76EFF2B2C3B3DAC
S31508007B605B5D00004552524F520A0D004F4B0A0DFD
S31508007B700000000044656661756C74004F70656EA0
S31508007B80424C5400FFF7FEBFFFF7FEBFFFF7FEBFEC
S31508007B90FFF7FEBFFFF7FEBFFFF7FEBFFFF7FEBF0B
S31508007BA0FFF7FEBFFFF7FEBFFFF7FEBFFFF7FEBFFB
S31508007BB0FFF7FEBFFFF7FEBFFFF7FEBFFFF7FEBFEB
S31508007BC0FFF7FEBFFFF7FEBFFFF7FEBFFFF7FEBFDB
S31508007BD0FFF7FEBFFFF7FEBFFFF7FEBFFFF7FEBFCB
S31508007BE0FFF7FEBFFFF7FEBFFFF7FEBFFFF7FEBFBB
S31508007BF0FFF7FEBFFFF7FEBFFFF7FEBFFFF7FEBFAB
S31508007C00FFF7FEBFFFF7FEBFFFF7FEBFFFF7FEBF9A
S31508007C10FFF7FEBFFFF7FEBFFFF7FEBFFFF7FEBF8A
S31508007C20FFF7FEBFFFF7FEBFFFF7FEBFFFF7FEBF7A
S31508007C30FFF7FEBFFFF7FEBFFFF7FEBFFFF7FEBF6A
S31508007C40FFF7FEBFFFF7FEBFFFF7FEBFFFF7FEBF5A
S31508007C50FFF7FEBFFFF7FEBFFFF7FEBFFFF7FEBF4A
S31508007C60FFF7FEBFFFF7FEBFFFF7FEBFFFF7FEBF3A
S31508007C70FFF7FEBFFFF7FEBFFFF7FEBFFFF7FEBF2A
S31508007C80FFF7FEBFFFF7FEBFFFF7FEBFFFF7FEBF1A
S31508007C90FFF7FEBFFFF7FEBFFFF7FEBFFFF7FEBF0A
S31508007CA0FFF7FEBFFFF7FEBFFFF7FEBFFFF7FEBFFA
S31508007CB0FFF7FEBFFFF7FEBFFFF7FEBFFFF7FEBFEA
S31508007CC0FFF7FEBFFFF7FEBFFFF7FEBFFFF7FEBFDA
S31508007CD0FFF7FEBFFFF7FEBFFFF7FEBFFFF7FEBFCA
S31508007CE0FFF7FEBFFFF7FEBFFFF7FEBFFFF7FEBFBA
S31508007CF012000120020102030404100706070809FE
S31508007D004D640008790412910452000112F30C1212
S31508007D10FD04830F651412210C100D0902200001C1
S31508007D200100C0320904000002FF1B200807058174
S31508007D30024000FF070501071003095900089F04C0
S31508007D401007B7580008EB5A0008810412CF04122E
S31508007D50B10410032F5B00083D04124B04126104A2
S31508007D6010075C00002039750008410412590412F6
S31508007D7049041269041279041289041002120110C6
S31508007D800161100340501DAC60751302030E100705
S31508007D9004030904A1770008A30412B50412B70462
S31108007DA012BF0412C70412D10403040128
S70508007B5126
